:020000040800F2
:1000000090100020B5810008BD800008BF80000866
:10001000C1800008C3800008C5800008CD810008A9
:10002000000000000000000000000000C780000881
:10003000C980000800000000CB800008CD800008C7
:10004000D1810008D5810008D9810008DD81000830
:10005000E1810008E5810008E9810008ED810008E0
:10006000F1810008F5810008F9810008FD81000890
:100070000182000805820008098200080D8200083C
:100080001182000815820008198200081D820008EC
:100090002182000825820008298200082D8200089C
:1000A0003182000835820008398200083D8200084C
:1000B0004182000845820008498200084D820008FC
:1000C0005182000855820008598200085D820008AC
:1000D0006182000865820008698200086D8200085C
:1000E0007182000875820008798200087D8200080C
:1000F0008182000885820008D1800008898200087A
:100100008D8200089182000895820008998200087B
:100110009D82000800000000A1820008A58200085E
:1001200000000000A9820008AD820008B18200082A
:10013000B5820008B9820008BD820008C1820008AB
:10014000C5820008C9820008CD820008D18200085B
:10015000DD800008D5820008D982000840F0200028
:1001600070472DE9F14FB0B0924604910DF1420174
:100170003A9A2B9199464A7000200AE01AF8011B1E
:100180000498309A90470028049000F041860D981A
:10019000401C0D909AF8000050B12528EED10021A6
:1001A00000220791089209910A920B910C9204E0A7
:1001B0000D9800F02FBE41F001011AF8010F202820
:1001C000F9D023280CD02B2804D02D2805D0302896
:1001D00009D00BE041F00201EFE741F00401ECE748
:1001E00041F00801E9E741F01001E6E72A280FD1C4
:1001F000D9F8002052F8040BC9F8002000280F900D
:1002000003D540420F9041F004010AF1010A14E0C5
:100210000F92DFF8083C0AE00F98984205DA00EBED
:10022000800402EB4402303A0F920AF1010A9AF874
:100230000020A2F130000A28EED39AF800002E2800
:1002400003D04FF0FF320E9229E01AF8010F2A284E
:1002500009D1D9F8000050F8042BC9F800000E921B
:100260000AF1010A1BE02D280CBF0AF1010A002047
:1002700000220E92DFF8A44B0BE040B90E9AA24286
:1002800005DA02EB820503EB4503303B0E930AF1DE
:10029000010A9AF80030A3F130020A2AEDD3ADF832
:1002A00040100FF67C309AF8001000F0FBFE08B109
:1002B0001AF8010B8DF842009DF84200682805D11C
:1002C0009AF8000068280CD1622106E06C2804BF6F
:1002D0009AF800006C2804D171218DF842100AF1BF
:1002E000010A12A806901AF801BBBBF125012CD017
:1002F0001C3900F09481091F022940F290811339C2
:1003000000F0B884093900F08A81891E00F04D851B
:10031000491E00F0FA84491E022940F28081091F1B
:1003200000F0F384491F00F0EF80491E00F0A28422
:10033000491E00F0D780C91E0CD0891E00F09A8497
:10034000C91E00F0978400F03BBD012307932521CF
:1003500000F033BDD9F8000050F8044BC9F8000094
:10036000002C059440F0AB802B994878002800F0D1
:10037000A1804FF0FF340FF6B02000F0ADFE241A3C
:1003800040F0468500F028BD01236A4602A93046A8
:1003900000F00EFE002840F03B85641EF4D130963C
:1003A000079C12AF74B1309E17F8011B0498B04738
:1003B0000028049000F02C850D98401C641E0D90C0
:1003C000F2D130960A9C3021002C8DF800100CDD03
:1003D000309E01236A4602A9304600F0E9FD00285C
:1003E00040F01685641EF4D13096059F089C74B1C8
:1003F000309E17F8011B0498B0470028049000F0C5
:1004000007850D98401C641E0D90F2D130960B9C10
:100410003021002C8DF800100CDD309E01236A463F
:1004200002A9304600F0C4FD002840F0F184641EAB
:10043000F4D1309605980899099C471874B1309EFC
:1004400017F8011B0498B0470028049000F0E084DE
:100450000D98401C641E0D90F2D130960C9C3021FA
:10046000002C8DF800100CDD309E01236A4602A995
:10047000304600F09DFD002840F0CA84641EF4D18F
:1004800030969DF8400041077FF584AE2020002D76
:100490008DF800007FF77EAE309C01236A4602A9EA
:1004A000204600F085FD002840F0B2846D1EF4D196
:1004B00030946FE60FF65830059000F08DBC0E9D1D
:1004C000002D04D5204600F027FE044607E02A460A
:1004D000204600F02BFE002814BF041B2C46089475
:1004E00000F07ABCD9F8001051F8040BC9F80010DC
:1004F00020F00004002121F0FF35CDE9024512ABC8
:100500000593782100F04DBC2B99487820B14FF02D
:10051000FF340FF6CC2030E79DF84200622860D00F
:10052000682817D06A283FD06C2806D0712847D099
:1005300074282CD07A281DD062E0D9F8001051F828
:10054000040BC9F80010002866D14FF0FF340FF6F5
:10055000A82012E7D9F8001051F8040BC9F80010D0
:1005600020B94FF0FF340FF6902006E70D99018077
:1005700000F032BCD9F8001051F8040BC9F8001093
:10058000002849D14FF0FF340FF66C20F5E6D9F87A
:10059000001051F8040BC9F8001000283CD14FF0AE
:1005A000FF340FF65420E8E6D9F8001051F8040B98
:1005B000C9F8001080B94FF0FF340FF63C20DCE69C
:1005C000D9F8001051F8040BC9F8001020B94FF009
:1005D000FF340FF62420D0E60D9AD317C0E900238C
:1005E000FAE3D9F8001051F8040BC9F8001020B94B
:1005F0004FF0FF340FF60020BFE60D990170EBE3DA
:10060000D9F8001051F8040BC9F8001020B94FF0C8
:10061000FF340FF6E410B0E60D990160DCE39DF8BD
:1006200042004C2807BFD9F80010CA1DD9F80000B5
:10063000C21D22F00702C9F80020D2E900010832E9
:10064000C9F80020CDE90201C80F02D007982D217A
:100650000AE0BDF84000810702D507982B2103E08E
:10066000C00705D50798202112AA1154401C0790F5
:1006700012A807994BF0200300EB010CDDE9020101
:10068000CDE92C01612BCDF814C021AC0BD00E9814
:10069000002848BF062105D404BF4BF0200067287E
:1006A00001D101210E91DDE902014F0047EAD07727
:1006B0007E15FF174FF0FF32974208BF964210D1C8
:1006C000090341EA10510003002908BF002808D09F
:1006D000ABF1610503211A2D089118D30FF63811DB
:1006E00010E0DDE902014A00521512F1010F11D1AB
:1006F00008030FD1ABF1610503211A2D08911FD317
:100700000FF61C110322604600F03CFD64E30FF677
:100710000411F7E7DDE902016A4600F03FFDCDE98B
:1007200002014BF02000612811D1059830210170A1
:10073000821C0592BBF1610F0CBF7821582102E0A9
:100740000FF6D801DEE741700798801C0790DDE9BD
:10075000020120F0000231F0004308BF002A02D15C
:100760000026002542E14BF02008B8F1610F40F06F
:1007700092800E98002847BF21210191401C0190D2
:10078000019FDDE92C017F1C00220023DDE90245E9
:1007900000F03CFD38BF85F0004500998DF88420BD
:1007A000091F002F00910DF1850632DD20462946F4
:1007B0000022002300F044FD2BD21C2200F05AFD41
:1007C00004460D4600F000FEFF1F002F804609DDA5
:1007D00000F01AFE02460B462046294600F0E4FED1
:1007E00004460D46F01D0721B8F1000F0CDD491E2F
:1007F0005EBF08F00F0200F8012D4FEA2818F3D56C
:1008000002E0002200F8012D491EFAD5C61D002F76
:10081000CCDC0DF18500361A01980DF18504864275
:10082000D8BF304600282FD4B04206DA0DF185013A
:100830000A5C082AA8BF0F2100DA0021024621AB7A
:10084000134400E0401E13F80159521E8D42F9D0A6
:100850000F2904D10DF185018B5C5B1C8B54002AA0
:1008600004D50099091D21AC401C0091411E0BD4F8
:10087000621813783033DDB23A2DA4BF5B443A3BA3
:10088000491E02F80139F4D50E99002940F1AC80D7
:10089000421E0E92A8E00099DFF8042747F2975015
:1008A000414391FBF2F20092DDE92C45C2F10702CF
:1008B000002A25F0004504DD2046294600F04CFBC7
:1008C0000BE052420020DFF8DC1600F045FB024648
:1008D0000B462046294600F0D9FE04460D46B8F1E5
:1008E000660F06BF009F0A3706270E983F18142F81
:1008F000C8BF142730208DF884000DF18506002F25
:1009000034DD2046294600F0E5FF01460A4606F19F
:10091000080304200A26B2FBF6F606EB860EA2EBCD
:100920004E02303203F8012C0A22B6FBF2F202EB3F
:10093000820EA6EB4E063036401E03F8026DE9D15A
:10094000083F002F03F10806D9DD084600F0D4FF68
:1009500002460B462046294600F026FE0022DFF81C
:10096000483600F0D7FF04460D46CAE70DF1850072
:10097000361A0DF1850404E00098401E761E0090A2
:10098000641C20783028F7D0B8F1660F02D10098A7
:10099000401C04E0B8F1650F0CBF012000200E9947
:1009A00040188642B8BF701E00281DD4B04204DA39
:1009B000215C3429C8BF392100DC30210246631E86
:1009C0009D1800E0401E15F80169521E8E42F9D0B4
:1009D000392902D1A15C491CA154002A04D50099EF
:1009E000491C1C46401C00910646009D01F088F8F9
:1009F000406A0778DDF8388030B2002802DC012632
:100A00000FF220644BF02000662808BF6D1C16D042
:100A1000672845D128B210F1040F47DB404545DA7D
:100A20009DF840006D1C010703D430B24045D8BF8B
:100A3000804628B2B8EB000848BF4FF000080FFA14
:100A400085FBBBF1000F00F3B4800898411C0891AE
:100A5000302205990A54B8F1000F03DC9DF84000DC
:100A6000010704D50898411C089105990F5418EB0B
:100A70000B0FB8BFC8F100052DB26842454432B231
:100A80000B909542B8BF2E46059B089836B2099642
:100A900032462146184400F075FBAD1B0C95D2E0A0
:100AA000BBF1610F17D14FF0700B19E030B2404528
:100AB00004DA9DF840100A0758BF8046B8F10108D3
:100AC00048BF4FF00008BBF1670F14BF4FF0450B54
:100AD0004FF0650B04E0BBF1410F08BF4FF0500B26
:100AE0000898411C0891B8F1000F059914F8012BE2
:100AF0000A5403DC9DF8400001071AD50898411CF0
:100B00000891B8F1000F05990F5412DD761E30B22E
:100B10008045B8BF46460598089B32B22146184426
:100B200000F030FB089936B271180891A8EB060066
:100B30000B9005980899084429B2002980F800B064
:100B400003D42B224270821C04E02D2242700D46F9
:100B5000821C6D4200212CAB28460AE004460A2084
:100B600094FBF0F000EB8005A4EB450403F8014B87
:100B7000491C00B20028F1DC012906DC4BF0200002
:100B8000652804BF302002F8010B00292CAB08D1E6
:100B9000302002F8010B06E0491E585C303002F8A4
:100BA000010B0029F8DC059908980844121A0992EB
:100BB00049E030B229B288421CDA0598089B32B26B
:100BC0002146184400F0DEFA089936B271180891EF
:100BD000ABEB0600B8F1000F0B9003DC9DF8400072
:100BE000020704D5059847540999491C0991CDF885
:100BF000308028E00598089B2AB22146184400F06E
:100C0000C1FA0898761B5844B8F1000F089003DC2D
:100C10009DF840100A0703D5411C089105990F540F
:100C200030B28045B8BF46460598089B32B204EB07
:100C30000B01184400F0A6FA089836B23018089054
:100C4000A8EB06000B909DF8400000F0140010285F
:100C500040F0C280079A08980B99821809988A1860
:100C600082180C980F998018884280F2B580081A73
:100C70000A90B1E09DF84200622808D068280ED0A2
:100C80006A2814D06C281FD0712810D01CE0D9F825
:100C9000001051F8040BC9F80010C0B21AE0D9F8DE
:100CA000001051F8040BC9F8001080B212E0D9F816
:100CB0000000C21D22F00702C9F80020D2E900019D
:100CC0000832C9F8002006E0D9F8001051F8040BEA
:100CD000C9F800100021CDE902019DF8400001078C
:100CE0005AD5DDE90223002B08BF002A54D04BF06F
:100CF0002000782850D1079812A930220A54401CAD
:100D0000431C079301F800B046E09DF842006228BA
:100D100008D068280ED06A2814D06C281FD07128FB
:100D200010D01CE0D9F8001051F8040BC9F80010DD
:100D300040B21AE0D9F8001051F8040BC9F80010BD
:100D400000B212E0D9F80000C21D22F00702C9F873
:100D50000020D2E900010832C9F8002006E0D9F8E5
:100D6000001051F8040BC9F80010C117CDE90201B9
:100D7000002902D507982D210AE0BDF8400081071F
:100D800002D507982B2103E0C00705D5079820213D
:100D900012AA1154401C079012A80799014405910A
:100DA000594602A800F04EF816E001200790D9F845
:100DB000000050F8041BC9F800008DF848100BE043
:100DC00001212522BBF1000F07918DF8482003D0A7
:100DD000022207928DF849B00F9D07990A986D1A63
:100DE00008992D1A0B986D1A09992D1A0C986D1ADD
:100DF0009DF840102D1A48073FF5D2AA2021002D5A
:100E00008DF800107FF7CCAA309E2C46FFF7BCBAB5
:100E10004FF0FF3031B0BDE8F08F0000CBCCCC0CF0
:100E2000686A6C747A4C00007072696E74665F73E5
:100E30003A2062616420257320617267756D656E6A
:100E4000740000002DE9FC4707468A463C6950467D
:100E50006F2808BF082505D0FFF780F9782814BF50
:100E60000A251025D7E900013C2680468946BAF1BB
:100E7000640F18BFBAF1690F05D1002903D5D8F165
:100E8000000869EB4909B9F1000F08BFB8F1000F7C
:100E90000CD1386B50B9082D3AD197F838000107BA
:100EA00036D530223B2684F83B2031E08DF800A077
:100EB000404649462A46EB1700F028FE3032D0B2B1
:100EC000761E3A2801960EDAA255404649462A4631
:100ED000EB1700F01BFE80465FEA010908BFB8F17E
:100EE000000F05D108E09DF800001218513AEBE719
:100EF000F868A1198842DBD3082D09D197F838008A
:100F0000010705D5A05D302802D0761E3020A055FF
:100F1000C6F13C03BB61A119F960386B834208DA62
:100F2000C31A3B624FF6EF70398F01403987BDE835
:100F3000F38700280ED597F8380000F01400102829
:100F400008D17A6B7969386A521A121AD21A002AB1
:100F5000C8BF3A62BDE8F3872DE9D04306460F4685
:100F600014464FF00008DFF8449012E0E00707D580
:100F700042464B463046394600F0CCFC06460F460A
:100F80004046494642464B4600F0C4FC6410804649
:100F90008946002CEAD130463946BDE8D0830000AE
:100FA000A08601000000F03F84D797410000244054
:100FB000F8B505460E4617461C4600205CB117F8EA
:100FC000011BB068A847B06030B1F06A401CF06205
:100FD0000020641EF3D1F2BD4FF0FF30F2BD0000DF
:100FE0007072696E74665F733A20256E206469734F
:100FF000616C6C6F776564007072696E74663A201C
:1010000062616420256E20617267756D656E740083
:10101000000000006E616E004E414E00696E660079
:10102000494E46003000F0B4024610689568131827
:10103000506803EB5004C00748BF4D44A3422DD075
:1010400013F8016B16F0030004BF13F8010BC01C6A
:1010500031090F2907D113F8011B0F3103E013F8F1
:10106000017B05F8017B401EF9D10029E6D013F879
:10107000010BC6F38106032E08BF13F8016B00EBCA
:101080000620404228440026B71E8F421EBF10F89B
:10109000017B05F8017B761CF6D1CFE7F0BC02F1AD
:1010A0000C007047C9B202788A421AB11CBF10F80E
:1010B000012FF9E718BF0020704703681AB95A1EBC
:1010C000026008467047197811B94FF0FF30704739
:1010D000591C01601878704780B500B906A0054911
:1010E0000B681BB122220021984701E000F091FD1E
:1010F000222002BD8C0C0020636F6E7374726169D4
:101100006E742068616E646C65723A20626164205E
:101110006D6573736167650000F1010310F8011BD1
:1011200011B110F8011BFBE7C01A7047C9B2830761
:1011300006D0521E22D310F8013B9942F7D11FE08E
:10114000083A13D302F1040241EA012141EA0141C4
:1011500050F8043B121F21BF4B40A3F1013C2CEA85
:10116000030C1CF0803FF3D0C9B2001F083210F806
:10117000013B521E28BF91EA030FF8D818BF012087
:10118000401E70474AB1000011F8013B521E00F8A2
:10119000013B1CBF11F8013BF8E7704710B514463E
:1011A00000F002F8226010BDC1F30A5343B14A00B7
:1011B00012F5001F28D2A3F2FE32A1EB02517047B4
:1011C00050EA410C20D001F0004C31EA0C01B1FA98
:1011D00081F204BFB0FA80F3D2180B3AB2F12003C7
:1011E0002CBF00FA03F1914041EA0C013EBFC2F16D
:1011F000200C20FA0CF319439040524240F2FD3388
:10120000D21A01EB035170470022704741EA030CE8
:1012100050EA4C0C52EA0C0C4FF4001C09D307D0D6
:101220001CEB410F9CBF1CEB430F8B4208BF82425B
:1012300070471CEB430FFBD8994208BF90427047A0
:1012400041EA030C50EA4C0C52EA0C0C4FF4001C1F
:1012500009D307D01CEB410F9CBF1CEB430F9942F5
:1012600008BF904270471CEB410FFBD88B4208BF70
:1012700082427047124254D440F2FF7C1CEA115360
:101280000FD0634531D09B1863453CBF01EB025141
:10129000704701F0004141EA0C510020AFF300809B
:1012A000704750EA410320D001F0004C91EA0C0154
:1012B0001CD0B1FA81F30B3B9A420DD9D21A994056
:1012C00051EA0C01C3F1200C20FA0CFC6144984057
:1012D000531C40F2FF7CD7E7914041EA0C01C2F178
:1012E000200C20FA0CF3194390407047B0FA80F3B9
:1012F0001533202BE0D3202AEED3203A203B9A420C
:1013000009D9D21A00FA03F141EA0C010020531C5A
:1013100040F2FF7CB8E700FA02F141EA0C0100203C
:101320007047524240F2FF7C1CEA11530DD06345D6
:10133000DBD0B2EB030C3CBFA1EB025170470CF1C8
:10134000010221EA035141F4801150EA410CCCD052
:1013500001F0004C352A27DC30B481EA0C01B2F1EF
:10136000200309DAC2F12003044601FA03F5D04054
:101370002843D1409C400CE0C3F12002450020FAF4
:1013800003F418BF44F0010421FA03F091400C4328
:10139000002174F1004550F1000051EB0C01244292
:1013A00030BC7FF47BAF70476146002076E78268EF
:1013B000521C8260426832B10268531C0360117093
:1013C0004168491E41607047C1F30A5340F21E4212
:1013D000D31A0CDDCA0283F3070342EA505242F0EB
:1013E0000042DA4002EBE17282EAE17070476FEA94
:1013F000E17203F2E13008B182F000407047026808
:10140000531C03601170704710F0004160B148BF79
:101410004042B0FA80F29040D21CC2F5846241EAA8
:10142000025202EBD021400570472E0070B491EAC1
:10143000030F4FF0004540F1BF806B40841A71EB01
:10144000030604D26E40001BB141121973414FF4E0
:10145000001C1CEB410F34BF7CEB430683E00C0DFA
:10146000A4EB1356362E00F37C80012E45EAC323ED
:1014700041DC43EA525312BFD20292025B082405B8
:1014800045EAC12141EA5051D2EBC020994125D40F
:1014900007D1B0FA80F610FA06F162D000202036AB
:1014A00008E0B1FA81F6B140C6F1200220FA02F25A
:1014B0001143B0404FEAF474B4EB465434F00106E3
:1014C0004FEA74040AD8D6F50016760D04F00044ED
:1014D000F04061FA06F25040F1404840C00A40EA4C
:1014E000415021F0004128BF5FEA500550F1000053
:1014F00044EBD12135E0DB0A45EAC121C90AB6F146
:1015000020050EDD42EA0242120CC5F1200603FA64
:1015100006F6EB4042EA06056D42984161F1000192
:101520000DE062FA06F5F240554063FA06FC82EAE5
:101530000C02F3405A406D42904161EB030111F4FB
:10154000801F05D1641E620502D06D0040414941F3
:1015500021F48011430875F1004350F1000041EB84
:10156000045170BC70471CEB410F15D223F00043AF
:1015700052EA43060BD04FEA4C0CBCEB410F04D8A7
:101580000C0D661E342EB7DDEBE7801A994150EA48
:10159000410608BF0021E4E708BF1CEB430F28BF4A
:1015A0006FF00001DDE7000070B491EA030F4FF027
:1015B00000457FF543AF6B40841A71EB030603D2FD
:1015C000001BB141121973414FF4001C1CEB410F79
:1015D00034BF7CEB430442E00C0DA4EB1356352ED4
:1015E0004FDC45EAC323DB0A45EAC121C912B6F143
:1015F00020050DDD63FA05F6EB4086EA030512428D
:1016000018BF45F00105C01851F100010CD213E0DC
:1016100062FA06F5F2405540F3415A40B340F340B8
:101620005A408018594107D349085FEA30005FEA01
:10163000350528BF45F0010501F58011420875F117
:10164000004250F1000041EB04514E0016F5001F1E
:1016500070BC38BF70470020090D090570471CEBAE
:10166000410F10D252EA43060BD0BCEB410F05D814
:101670000C0DAB43661E342EB6DD02E0AB43801882
:10168000594170BC704770BC70474300F0B540F2E0
:10169000FF7581EA030C0CF0004C15EA11541DBFD4
:1016A00015EA1357AC42AF42E5E0BC41C1F3130168
:1016B000C3F31303801A994143F4801304D2641EC8
:1016C0000018494180185941C90241EA5051B1FB03
:1016D000F3F603FB1611A2FB0675D7EBC020A94158
:1016E00002D2761E80185941C90241EA5051B1FB1D
:1016F000F3FE03FB1E11A2FB0E75D7EBC020A94120
:1017000003D2AEF1010E80185941890241EA90518D
:10171000760546EA8E2EB1FBF3F603FB1611A2FB0B
:101720000675D7EB8020A94102D2761E8018594158
:10173000C90241EA50514EEA060EB1FBF3F603FB33
:101740001611A2FB0675D7EBC020A94102D2761E66
:1017500080185941C90241EA5051B1FBF3F703FB2C
:101760001711A2FB0735D3EBC020A94167F1000791
:101770000CBF004247F0010766F3D5274FEA1E3140
:10178000B80814F5806412DDBD0775F1004250EB16
:101790000E5051EB045111F5801F5CBF41EA0C0162
:1017A000F0BD4CF07F6141F0E0410020F0BDBD078D
:1017B0006D0840EA0E5041F48011D4F10104B4F1F7
:1017C00020060ADAC4F120060200E04001FA06F31E
:1017D000E1401843B24015430EE0342C13DCC6F14F
:1017E000200445EA40056D0820FA06F2154321FA67
:1017F00006F0A1400D43002175F1004250F10000B8
:1018000051EB0C01F0BD00205FEA0C01F0BDCFB937
:1018100092185B41B3FA83F704BFB2FA82F6BF199C
:101820000B3FB7F120062FBF02FA06F3BB40C7F10A
:10183000200622FA06F638BF3343BA401CB1E41939
:10184000641E33E77F4231F00041B1FA81F404BFF6
:10185000B0FA80F6A4190B3CB4F120062FBF00FAB1
:1018600006F1A140C4F1200620FA06F638BF314344
:10187000A0403C1B1AE7AC421ABF05EA1357AF421F
:1018800012E050EA41061CBF52EA4306BFE750EAA5
:101890004107304661461CBF41EA0551F0BD52EA9E
:1018A000430C08BFC143F0BD00204FF4001616EBF7
:1018B000410F98BF16EB430F08BF16EB410F24BF33
:1018C000C14305E016EB430F0CBF61464CEA0551DE
:1018D000F0BD0000400D40F21E4C40EAC120BCEBC0
:1018E000115C40F0004003D48CF30701C8407047FE
:1018F0006FEAE1707047000050B1B0FA80F18840A3
:10190000C91CC1F58461090501EBD0214005704770
:101910000146704730B540F2FF7C1CEA11541DBFF0
:101920001CEA1355644565453FE0641981EA030CE0
:101930006FF35F530CF0004C43F48013C90241F085
:10194000004141EA505EC5021100A5FB02020028D9
:101950004FF00000EEFB01204FF00001E3FB0521FA
:1019600018BF42F00102401800214941E3FB0E017B
:10197000A4F580640D0302D292184041494154F10C
:10198000010470DD450872F1004250F1000051EB96
:101990000451A1F5801102D441EA0C0130BD40F29E
:1019A000FF7E4CEA0E51002030BD0CEA1355644511
:1019B00018BF654581EA030C0CF0004C41D050EA99
:1019C000410E1CBF52EA430E02E06146002030BDCA
:1019D00024422C441BD15FEA050EF6D0090302BF56
:1019E00001460020AEF1140EB1FA81F5AEEB05040C
:1019F00001FA05FE0C35C5F1200100FA05F5C840D5
:101A00004EEA000E6FF35F5343F480139CE733F00C
:101A10000043B3FA83F504BFB2FA82FE75440B3D6E
:101A2000641BB5F1200E2FBF02FA0EF3AB40C5F1D7
:101A3000200E22FA0EFE38BF43EA0E03AA40641CB1
:101A40007CE750EA410E14BF52EA430E6FF00001EA
:101A50004FF4001515EB430F8EBF194615EB410FE0
:101A60009DE7B4D830BDD4F10104B4F120050FDAFC
:101A7000C4F12005520828BF42F0010210FA05FE09
:101A800001FA05F57244E2BFE0402843E1400FE06F
:101A9000352C9ADCC5F1200452EA400220FA05F206
:101AA00018BF42F0010231FA05F0A1400A430021BB
:101AB00072F1004250F1000051EB0C0130BD00000A
:101AC000613807E005E0A0F161011A2901D2012087
:101AD000704741381A288041C00F7047A0F10901B2
:101AE000052901D3202801D101207047002070472B
:101AF000A0F141011A2938BF2030704701487047D2
:101B0000014870474800002010000020D3BBD9B125
:101B1000B2F5803F5BD2022A1ED98C46B1FBF2F1AE
:101B200002FB11C31B0443EA1043B3FBF2FC02FBAC
:101B30001C3380B240EA0343B3FBF2F002FB1032E5
:101B400040EA0C4000237047022A05D98446B0FBC6
:101B5000F2F002FB10C270474AB105D100F0010259
:101B600049085FEA3000704700220023704700F008
:101B700053B80B000200002100207047F7D3002269
:101B800000237047904271EB030CF2D370B5B1FAA9
:101B900081F4B3FA83F52C1BA340C4F1200532FA7B
:101BA00005F63343A2405FF00046E64002E05B08E2
:101BB0005FEA3202841A71EB030524BF20462946EE
:101BC0007641F4D302000B003000002170BD70B5E7
:101BD000B1FA81F4B2FA82F5C4F120046419B4F1C7
:101BE0002006DAD3B2405FF00044F440002502E062
:101BF00052085FEA3303C61A71EB020E24BF304667
:101C0000714664416D41F3D302000B0020002900AE
:101C100070BD012000F002B87047000080B5AFF33E
:101C20000080024A11001820ABBEFBE7260002002C
:101C300038B5040001D1012032BD04F18405686883
:101C400008B900F017F800F01AF808B100F031F800
:101C500000F02CF8012804D000F004F821F02A014B
:101C600016E032BD2068416821F49041416020684F
:101C70008168704700212970204600F082BF24202F
:101C8000686020680168490849000160A06A7047DF
:101C9000816000F004F8BDE8324000F0AFBB20687E
:101CA000016841F00101016020467047204600F0C4
:101CB0002DBA204600F03FBB38B5040001D1012009
:101CC00032BD04F184052420686000F014F8226815
:101CD0000020002110602368596021688860204638
:101CE00000F0E0FF0020E86000216960A860E16684
:101CF0002067297032BD20680168490849000160E9
:101D000070472DE9F843054605F15406706B0C4603
:101D10001746994620283ED10CB1380001D1012048
:101D20003AE00020F0632121716301F06DF8378003
:101D300080467780A868B0F5805F04BF28690028D6
:101D40001ABF204600272746044611E000228021C2
:101D500000F024F8D8B92868002C12BF14F8011B31
:101D600037F8021BC1F3080181627088411E71803F
:101D70007088CDF8009043460028E7D1002240212A
:101D800000F00CF818B920207063002004E0202037
:101D90007063032000E00220BDE8F283284600F0D3
:101DA00074BB38B50346D3F88C0020280AD109B19A
:101DB000100001D1012032BD00F006F8BDE8384026
:101DC00000F0ABBB022032BD0020D8661868DFF8F7
:101DD0003843A0420CD04068040209D5186850E886
:101DE000004F054644F0806445E800400028F5D1E6
:101DF0001846704728688168480670472DE9F04109
:101E000005462A68D36940F60F0610460768D2F8DF
:101E1000088005F15C0407F0200003F02001334244
:101E20000ED1002914D018B95FEAC80040F18780AC
:101E3000A169002900F02F812846BDE8F04108473C
:101E4000DFF838C818EA0C0F04BFDFF834683742EF
:101E500075D0DE0709D5FE0507D54FF0010EC2F893
:101E600020E0626B42F0010262639A0748BF5FEABA
:101E7000C87206D52E6802223262626B42F00402FA
:101E800062635A0748BF5FEAC87206D52E6804220B
:101E90003262626B42F0020262631A070DD50028BB
:101EA00008BF18EA0C0F08D0D5F800C00822CCF8FB
:101EB0002020626B42F0080262631A0509D57B019B
:101EC00007D52F684FF400623A62626B42F020023D
:101ED0006263626B002A31D039B110B95FEAC80081
:101EE00003D5A16909B128468847606B29688A68CB
:101EF000510602D410F0280F1BD000F0D4F8FFF7E1
:101F000079FF11D500F0D2F8FCD1606A60B10FF210
:101F1000A171C166606A00F0BBFF00280ED0606A44
:101F2000C16EBDE8F04108472846BDE8F04100F029
:101F3000D0BF284600F0CDFF00206063ABE02069F1
:101F4000012875D1D80673D5F90671D51020106215
:101F50002A6821889068420632D5626A1068806CCF
:101F600080B2002823D0884221DA6080106D812859
:101F700016D000F0B4FCFCD100F0B8F8FCD100F0B1
:101F8000A8F8FCD1202020630021216100F09CF8FA
:101F900021F0100100F083F8F8D1606A00F03AFFF8
:101FA0000220606121886088091A89B206E08842AF
:101FB00004BF106D81286ED102226261284633E091
:101FC00062886088891A00281CBF88B2002862D005
:101FD0002A46106850E8003F054623F4907345E810
:101FE00000300028F5D1106800F1080353E8003FE5
:101FF00000F10808DFF82C03034048E8003000280F
:10200000F1D12020206300232361A361136853E8EA
:10201000003F156823F0100345E800300028F5D193
:102020000220606189B21046BDE8F04100F052BF65
:1020300018060AD5390658BF5FEA082005D5E169B8
:1020400049B32846BDE8F0410847580611D579063E
:102050000FD500F039F821F0400100F020F8F8D158
:102060002020E0620021E1612846BDE8F04100F057
:1020700032BF180206D5790004D52846BDE8F041E4
:1020800000F02ABFD80148BF002F04D52846BDE87C
:10209000F04100F022BFBDE8F08141F4807142E8D8
:1020A000001000287047284600F0BDBA296801F1E9
:1020B000080252E8001F286800F1080321F04001DF
:1020C00043E8001000287047286850E8001F0246C7
:1020D0007047286800F1080151E8001F00F108036B
:1020E00021F0400143E8001000287047286800F103
:1020F000080151E8001F00F108034908490043E8BE
:10210000001000287047000000240046F8B504467F
:102110002268DFF8F40600251368A16803402069EF
:102120000B4361690343E0690B4303431360516848
:10213000E06821F4405101435160DFF88417A3693E
:102140008A421CBF206A03439668DFF87807DFF8ED
:1021500078E7064033439360D36A606A0FF25C56B7
:102160001B0940EA0313DFF86407DFF86477D362E2
:102170004FF4004372453AD13F6807F00307032F3D
:102180005AD8DFE807F0025350564FF0010CE169CE
:102190004FF6F077B1F5004F40F09080BCF1000FA2
:1021A0000FD0BCF1010F00F08180BCF1040F0CD006
:1021B000BCF1080F00F07D80BCF1100F00F07C80B6
:1021C000A5E001F0ADF9002810D000F0ADF84A0804
:1021D00002EB4002B2FBF1F0A0F11001B942EFD2E4
:1021E0000740C0F3420007432068C76090E0DFF873
:1021F000A4C762450CD13F6817F00C0706D0042F26
:1022000014D0082F0FD00C2F13D015E0AC46BEE72A
:102210008A4211D1BF6807F00307032F0CD8DFE80B
:1022200007F01C0502084FF0040C07E04FF0080C03
:1022300004E04FF0100C01E04FF0200C8A42A6D1D0
:10224000BCF1020F09D0BCF1040F0AD0BCF1080F99
:1022500015D0BCF1100F15D059E001F06FF900282E
:1022600056D0616A36F81120B0FBF2F6626802EBD4
:1022700042018E424BD31303B34205D247E001F033
:1022800030F9ECE71846ECE75008002110EB062087
:10229000DFF8A87751EB16610023FFF737FCA0F5B4
:1022A0004076BE4233D22168C86031E001F03DF98A
:1022B00089E701F016F986E7184686E7BCF1000FBA
:1022C0000CD0BCF1010F1AD0BCF1040F09D0BCF145
:1022D000080F17D0BCF1100F17D018E001F020F94B
:1022E000B0B100F021F800EB5100B0FBF1F0A0F12B
:1022F0001001B9420BD2226880B2D06008E001F030
:1023000014F9EDE701F0EDF8EAE71846E9E70125F1
:1023100004F168000121002341800180C360036152
:102320002846F2BDFEFFFFEF626A616836F81230A0
:10233000B0FBF3F0704790F828100A0706D5026842
:102340005368816B23F400430B43536090F82810CB
:10235000CA0706D502685368C16A23F400330B43E9
:10236000536090F828108A0706D502685368016BFD
:1023700023F480330B43536090F828104A0706D5A6
:1023800002685368416B23F480230B43536090F839
:102390002810CA0606D502689368C16B23F48053DF
:1023A0000B43936090F828108A0606D5026893685C
:1023B000016C23F400530B43936090F828104A06F5
:1023C00010D502685368416C23F480130B435360AB
:1023D000436CB3F5801F05D15368816C23F4C003AF
:1023E0000B43536090F828100A0606D501684A6826
:1023F000C06C22F4002202434A607047F8B50546DB
:1024000005F184040020E06000F0FEFC0646286828
:102410006FF07E4701680A0711D500973346002206
:102420004FF40011FFF7BAFC48B1FFF74DFE21F061
:102430008001FFF734FEF8D12020606017E02868A3
:1024400001684A0717D50097334600224FF48001F0
:10245000FFF7A4FC78B1FFF737FE21F49071FFF786
:102460001EFEF8D1FFF742FEFCD12020A060002123
:1024700021700320F2BD202060602021A160002097
:10248000E866002129672070F2BD2DE9F04105467C
:102490000E4690461F46069C2868C1693140B142ED
:1024A0000CBF01200020404535D114F1010FF3D0BD
:1024B00000F0AAFCC01B844200D314B90320BDE87D
:1024C000F081286801684A07E6D5802E18BF402EA3
:1024D000E2D0C169080704D42968C8690105DBD5C1
:1024E0000CE02A6808201062FFF7DDFD05F184008A
:1024F0000821C160002202700120E0E729684FF442
:1025000000600862FFF7CFFD05F184002021C16063
:1025100000220270D2E70020D1E750B5034699654A
:1025200003F15C010A804A80002088619868FF24DA
:10253000B0F5805F04D1186990B940F2FF140FE044
:1025400018B9186960B17F2007E0B0F1805F06D14B
:10255000186908B97F2403E03F20888001E0002447
:102560008C800020486322240C63186800F098F8DF
:1025700044F0010446E800400028F6D18868B0F134
:10258000005F21D1888982421ED39A68B2F5805FAC
:1025900004BF1869002803D10FF259328A6109E09B
:1025A0000FF27D248C61186920B100F02FF8FFF73D
:1025B00074FDFAD100F02FF841F0805144E800108A
:1025C0000028F7D1002050BD9868B0F5805F04BFA7
:1025D000186900280CD10FF24D128A61186850E872
:1025E000001F024641F02001FFF759FDF6D1E9E74F
:1025F0000FF2E1028A6118690028EFD000F006F8B6
:1026000041F49071FFF74BFDF8D1DBE7196851E811
:10261000001F1A687047186800F1080151E8001F90
:1026200000F10804704710B500F00EF8FCD100F07E
:1026300015F8FCD1C16E00F025F82021C0F88C10EF
:102640000022C266426710BD016851E8002F0B46A8
:1026500022F4907243E8002100297047016801F1DB
:10266000080252E8002F01F10804DFF844140A4080
:1026700044E800210029704700000000010000101C
:1026800020010004012909D1026852E8002F0368E3
:1026900022F0100243E800210029F5D170471068AC
:1026A00000F1080454E8004F00F1080670470000EC
:1026B000C06D0021A0F85E1000F00BBC010002000C
:1026C0000400060008000A000C0010002000400072
:1026D0008000000138B500F04DF81ED14B6A91889A
:1026E000846D0B402370816D4B1C00F049F818D1AC
:1026F00000F04DF800F060F8FCD100F06AF80BD162
:102700000023136100F04EF8FCD10168CB69DC06B0
:1027100044BF10230B6279E07DE0886940F0080037
:10272000886131BD38B500F025F81ED14B6A91881B
:10273000846D0B402380816D8B1C00F021F818D133
:1027400000F025F800F038F8FCD100F042F80BD189
:102750000023136100F026F8FCD10168CB69DC0688
:1027600044BF10230B6251E055E0886940F0080037
:10277000886131BD00F15C020168136B222B704748
:10278000836551884B1E5380518800297047036828
:1027900053E8003F046823F4907344E800310029B3
:1027A000F5D17047016851E8003F0C4623F0100353
:1027B00044E8003100297047016801F1080353E83B
:1027C000003F01F108055B085B0045E80031002986
:1027D000704720211163002393610021516101683A
:1027E000374B99420CD049680B0209D5016851E872
:1027F000003F0C4623F0806344E800310029F5D106
:102800001169012970470000F369FFCF1188BDE805
:10281000344000F05FBBBDE8324000F0B3BA0000C6
:102820002DE9F84300F00CF946D1A089002835D0F5
:10283000B80633D500F0B0F80870A86D421C00F05F
:10284000D9F812D0F90748BF5FEAC85200F0AAF8D9
:1028500003D5F10701D500F0C5F800F0ACF820B1C0
:10286000284600F036FB0020606360880028DFD136
:1028700000F035F8FCD100F0D3F8FCD100F0FEF800
:1028800009D100F0EBF844BF1021016221882846ED
:1028900000F020FB02E0284600F074FA608868B17E
:1028A000A18988420ADA00F0AEF8FCD18148A06123
:1028B00000F08EF8FCD101E000F00CF8BDE8F183E7
:1028C00000240046FFF4FF11003801400024F4000A
:1028D000E00C0246816941F0080181617047296876
:1028E00051E8001F2A6821F4807142E80010002896
:1028F000704700002DE9F84300F0A2F846D1A08906
:10290000002835D0B80633D500F046F80880A86D09
:10291000821C00F06FF812D0F90748BF5FEAC85276
:1029200000F040F803D5F10701D500F05BF800F0A6
:1029300042F820B1284600F0CCFA0020606360889D
:102940000028DFD1FFF7CBFFFCD100F069F8FCD104
:1029500000F094F809D100F081F844BF1021016221
:102960002188284600F0B6FA02E0284600F00AFA6C
:10297000608868B1A18988420ADA00F044F8FCD185
:102980004D48A06100F024F8FCD101E0FFF7A2FF60
:10299000BDE8F183004400402968486AA96D09EA4E
:1029A0000000704705D501210162606B40F0010015
:1029B0006063B8077047780708D5F10706D52A681D
:1029C00004201062606B40F002006063606B70472F
:1029D000296851E8001F2A6841F0200142E80010F0
:1029E000002870472A6802201062606B40F00400E3
:1029F00060637047AA656088411E61802868C76966
:102A000017F0070F7047286800F1080252E8001F0E
:102A100000F1080921F0805149E8001000287047B2
:102A2000286800F1080151E8001F00F10803204860
:102A3000014043E8001000287047000000FD0F002F
:102A40000546286805F15C04B4F80490C76901469E
:102A5000D1F800808668216B22297047002121610E
:102A6000286850E8001F024621F0100142E80010DB
:102A70000028F5D12868C169CA0670472020206364
:102A80000021A1610020606128680C4988420CD0B7
:102A90004068010209D5286850E8001F024621F06D
:102AA000806142E800100028F5D1206901287047B4
:102AB000FEFFFFEFD526000825270008002400466A
:102AC00010B5DFF81C43DFF81C0300F04EF822625B
:102AD0006262A26262662046FFF7AAF808B100F0BF
:102AE00013FE0021204600F037FE08B100F00CFE76
:102AF0000021204600F03BFE08B100F005FE204614
:102B000000F00CFE18B1BDE8104000F0FDBD10BD96
:102B100010B5DFF8D442DFF8D40200F026F8E26105
:102B200022626262A2622046FFF782F808B100F0DA
:102B3000EBFD0021204600F00FFE08B100F0E4FD9F
:102B40000021204600F013FE08B100F0DDFD204614
:102B500000F0E4FD08B100F0D7FDA54901F2DC501A
:102B600000220260204601221CE120600C204FF46C
:102B7000E131002260616160A260E2602261A261D5
:102B8000704770B596B004461421684600F042FEC6
:102B9000402106A800F03EFE20689249954C964DD3
:102BA000964E884223D14FF40072002106920F9175
:102BB00006A800F033FE08B100F0A6FDF06940F071
:102BC0004000F061F06900F0400000F05AF84FF466
:102BD000006100F04DF8082100F043F800224FF4A6
:102BE000806000F033F8082200F036F82CE07F49CE
:102BF000884229D1012200210692079106A800F0FF
:102C00000DFE08B100F080FDB06940F48040B06175
:102C1000B06900F4804000F034F84FF4805100F0C7
:102C200027F8072100F01DF800224FF4807000F013
:102C30000DF8072200F010F8002200212E2000F0ED
:102C4000FEFE2E2000F022FF16B070BD022102927F
:102C5000039200900191704704926946204600F06B
:102C600075BF0222049101926946284600F06EBFAA
:102C700002F0010205920598009100210291039152
:102C8000704705900598316841F002013160326863
:102C900002F0020205920598316841F001013160AD
:102CA0003268704738B501684E4B554A514C52480E
:102CB00099420ED155684FF4006125F040055560EA
:102CC00000F0FBFF20464FF48061BDE8344000F087
:102CD000F4BF464B994211D1116821F48041116033
:102CE0004FF4805100F0E9FF4FF48071204600F06E
:102CF000E4FF2E20BDE8324000F0D3BE31BD38B530
:102D00000446394D2846FEF7D7FF6C602846FEF78B
:102D10008FFF10B14FF0FF3032BD3A480021016003
:102D2000002032BD10B5324C40F2DC51204600F09C
:102D300071FD04F2DC500022026010BD0A4601461B
:102D400080B54FF0FF332848FEF7DBFF08B14FF0A6
:102D5000FF3002BD264910B501F2DC5253881488B9
:102D6000A3420CD0C95C0170508840F2DC51401C79
:102D700083B28B42A8BF00205080002010BD4FF0CE
:102D8000FF3010BD10B51A49B1F8DC3540F2DC5403
:102D90005B1C9AB2A242A8BF0023A1F8DC359BB20B
:102DA00001221944BDE81040FEF7FBBFF8B50C4600
:102DB0001546012818BF022802D04FF0FF30F2BD9F
:102DC0000026074F07E04FF0FF330122A1193846D4
:102DD000FEF797FF761CAE42F5D32846F2BD000001
:102DE000E00A002000240046740B00200038014057
:102DF000D800002000000242000402428C0C02466F
:102E0000A40C0246B406002001484068704700BF89
:102E10000000002070B50446FFF7F6FF06462CB30D
:102E200004F14C05287A022802D02021E9601BE039
:102E30002068416941F00401416105202872206841
:102E400001698A0414D4FFF7DFFF801B0628F6D33C
:102E5000E868032140F01000E86029722879010633
:102E600002D5A96A0120087300202870012070BDD6
:102E7000416941F0020141610420287222684FF447
:102E8000FE410120D16000F018F80020287070BDCC
:102E900030B100F154010A78022A03D020204860A2
:102EA0000120704704220A700068416941F4005112
:102EB00041F0040141610020704728722979080619
:102EC00005D5A86A01210173226800219164704729
:102ED0000000704770477047704770472DE9F84F02
:102EE000040044D0DFF80477D7F81C90D7F828A066
:102EF000207809F00C090AF00305C1072AD5B9F1B9
:102F0000080F04D0B9F10C0F08BF032D62D160681F
:102F100000282CD0B9F1080F1CD13968A068012213
:102F200021F48811014341F4803139603868DFF8B9
:102F3000DC16DFF8D436000D00F001008240B1FB52
:102F4000F2F1DFF8C0261160186800F029FF0028B0
:102F500040F0E9812078810712D5B9F1000F04D043
:102F6000B9F10C0F08BF022D57D12069002800F0DD
:102F7000DA813869616920F4F81040EA014038616B
:102F80002078DFF88C86DFF88C56010740F1C0808E
:102F900028684FF0000A41070AD428684FF0010A58
:102FA00040F004002860296801F0040100910098B5
:102FB000D8F80010C80751D400F0DDF90646D8F85B
:102FC0000000C1074AD4FFF71FFF801B0328F6D378
:102FD00003207FE1606888B13A68A16822F4881212
:102FE0001043084300F0C4F9064638688103B1D4A1
:102FF000FFF70AFF801B6528F7D3E9E7386820F45C
:10300000881000F0B5F9064638688103A2D5FFF7AD
:10301000FBFE801B6528F7D3DAE7206978B13968B1
:1030200041F480713960FFF7EFFE054638684105CD
:103030009FD4FFF7E9FE401B0328F7D3C8E73868A1
:1030400020F4807000F094F905463868410597D562
:10305000FFF7DAFE401B0328F7D3B9E7EE6DA0694E
:10306000002843D040011AD5E16906F08050814222
:1030700011D031010FD526F08066EE65FFF7C4FE52
:103080008346E86D010106D5FFF7BEFEA0EB0B00FD
:103090001528F6D39CE726F08050E6690643A06920
:1030A0000643EE65FFF7B0FE0090B346A669E86DF3
:1030B00010EA460F06D1FFF7A7FE0099401A15281F
:1030C000F4D385E786F010562BEA060BC5F85CB002
:1030D000FFF79AFE8346E86D10EA460F16D0FFF719
:1030E00093FEA0EB0B001528F5D371E726F01056E0
:1030F000EE65FFF789FE0646E86D10F0904F05D0AB
:10310000FFF782FE801B1528F6D361E700F028F94F
:10311000217848076CD529684FF0000A48070AD47F
:1031200029684FF0010A41F004012960286800F085
:10313000040000900098D8F80010C8070CD400F0E4
:103140001AF90646D8F80000C10705D4FFF75CFE5F
:10315000801B0328F6D33BE7E06841F2893828B3A7
:10316000E96D21F080010843E865FFF74DFE064652
:10317000E86D810705D4FFF747FE801B4045F7D374
:1031800026E7207B010608D5E86D01052ED4FFF760
:103190003BFE801B4045F7D31AE7E86D010525D5B6
:1031A000FFF732FE801B4045F7D311E7E86D20F0B2
:1031B0008100E865E86D20F00400E865FFF724FE73
:1031C0000646E86D810705D5FFF71EFE801B4045CA
:1031D000F7D3FDE6E86D010608D5E86D010505D5D4
:1031E000FFF712FE801B4045F7D3F1E600F0B8F878
:1031F000206A00286DD0B9F10C0F6DD00228386814
:1032000020F08070386053D1FFF7FEFD0546D7F8F7
:1032100000A0FFF7F9FD401B0328E6D25FEA8A1001
:10322000F5D4626A032A07D14FEA1A51DFF8DC03AA
:1032300001F00101C84001E0DFF8C403A36ADFF830
:10324000D813B0FBF3F088422CBF0C210021D7F833
:103250002890DFF8C8035B1E00EA0900024311430F
:1032600041EA032141F48021B962E06A216B401EEA
:10327000491E40EA4120616B491E40EA0140A16BB2
:10328000491E40EA01607863E06B10B100F062F81B
:10329000B862386840F0807000F06AF80446386818
:1032A000810116D4FFF7B0FD001B0328F7D38FE68A
:1032B000FFF7AAFD04463868810105D5FFF7A4FD94
:1032C000001B0328F7D383E6B86ADFF854130840DD
:1032D000B8620020BDE8F28F012824D0B86A796B6B
:1032E000636A00F003029A4201BFC0F30220401C4F
:1032F000A26A904217D1E26AC1F30800401C9042D2
:1033000001BFC1F34620401C226B90420BD1626B7F
:10331000C1F30640401C904201BFC1F30660401C4F
:10332000A16B884201D00120D4E7B86BE16BC0F3F8
:10333000CC008142CDD0B86A20F01000B862FFF70F
:1033400063FD0546FFF760FD401BFBD0E06B00F01E
:1033500001F8BDE7C000B863B86A40F010007047DC
:10336000BAF1000F03D0286820F0040028607047ED
:103370003860FFF749BDD8F8001041F00101C8F8E6
:103380000010FFF741BD2DE9F0410400884637D019
:10339000DFF89052286800F00F00404509D22968F4
:1033A000090948EA01112960286800F00F0040452A
:1033B00026D12178880609D5DFF840221368A16953
:1033C000E06923F017030B43034313602178DFF810
:1033D0001C72C80742D53868616803290CD1800186
:1033E0006BD5F96901F00C010C290CD0B96A0120E8
:1033F00060F31551B96206E0022902D1800302D4BC
:103400005BE0410559D5FA696068920840EA82029A
:10341000FA61FFF7F9FC06466068F96901F00C01F2
:10342000B1EB800F08D0FFF7EFFC801B41F2893130
:103430008842F1D3032052E003280FD1B86A20F468
:103440008010B862FFF7E0FC0646B86A410205D476
:10345000FFF7DAFC801B0B28F7D3EBE7396A226809
:103460000020930704D5C908C800A16801430120C2
:10347000530704D521F07000E168014301201207D1
:1034800005D5206921F4E06141EA001100E000B1B6
:1034900039622078C10644BF60697862296801F00A
:1034A0000F0188450BD22868000948EA00102860FF
:1034B000296801F00F01414501D001200FE000F023
:1034C00010F83A6A58494F4B02F00702895CC8402D
:1034D00018604D480068BDE8F04100F061BCBDE8EF
:1034E000F0814249C86910F00C0001D1444870478E
:1034F000082818BF00F036B809684448090D01F0E3
:103500000101C840704780B5FFF7EBFF47490968E4
:10351000454A3C4B01F00701515CC840186002BDB0
:1035200080B5FFF7F0FF414A0CE080B5FFF7EBFFF5
:103530003E4A13683E49C3F3022207E080B5FFF715
:10354000E2FF3C4A13683A49C3F30212895CC8405F
:1035500002BD10EE100A491CB0FBF1F010BD364858
:10356000046807E010B5FFF7FAFFBCEEC00AC4F329
:103570000661EEE71D48416BC1F30801491C00EEEE
:10358000101A816AB8EE400AC1F30222521C00EE02
:10359000902AF8EE600ACA0643BF826BC2F3CC02DF
:1035A00001EE102A9FED121A01F00301B8EE411A44
:1035B000022902D0032903D00DE0DFED0E1A0CE042
:1035C00000681249000D00F00100C14001EE901AA0
:1035D000F8EE611A01E0DFED061AC1EEA00ADFED98
:1035E000061A01EE210A20EE800A7047000C0246FE
:1035F000000000000024744B00000039000E024659
:103600000024F4000C000020080000200048E8011D
:1036100028080246940C024601127A00E0F8FFFFE7
:10362000FCFFF8FF0020024098470008200C0246EB
:10363000C4810008240C0246340C024610B500F088
:10364000F9FB00F01DF800F00FFCFFF739FAFFF767
:103650005FFA00F0ABFC00F007FD00F015FD074C31
:1036600000280CBF204604F1240000F0BBFF00F04E
:1036700070FC00BF25A000F0B5FFFEE7BC7D000890
:1036800080B598B0402108A800F0C4F82021684611
:1036900000F0C0F84FF4803000F0B8FF08B100F03F
:1036A00033F800220A920F924FF4803103220991DD
:1036B00011924FF08061082209200E911392089018
:1036C00002210022109112911491159116911792D6
:1036D00008A8FFF703FC08B100F016F83F2100919D
:1036E00000210322029104910192042100220691FB
:1036F00003920592079201216846FFF744FE08B144
:1037000000F002F819B000BD72B6FEE74C54452037
:103710005445535420444F4E450D0A0010B500F156
:1037200084010A78012A01D1022010BD01220A7009
:1037300024234B60026813681468640864001460F2
:1037400000224266006823F00053202203604A6092
:1037500000230B70002010BD70B500F01FF801D1E0
:10376000022070BD00F020F822F0604209E070B540
:1037700000F014F801D1022070BD00F015F822F01D
:10378000606211438160204600F01CF8206820210F
:103790000022066069602A70002070BD044604F1B2
:1037A00084052878012870470120287024226A6047
:1037B0002068066802685208520002602068826829
:1037C0007047000030B5416E11B90121012214E0AB
:1037D000016800BF0FF22C040CA38A688968520E9E
:1037E00002F00702490F655CA45C595C9A5CED002D
:1037F000E40095FBF1F194FBF2F268304180028025
:1038000030BD0000010101030701000008040204AB
:1038100008010101002200F027BF00002DE9FC474C
:1038200006463078DFF8EC71C10705D53A68706854
:10383000920840EA82023A603178880705D53968F3
:10384000B06821F00C01014339603178480705D593
:103850003968F06821F44061014339603178080724
:1038600005D53968306921F4402101433960317848
:10387000C80605D53968706921F4401101433960E3
:103880003178880605D53968B06921F440010143D3
:1038900039603178480605D53968F06921F0004172
:1038A000014339603168DFF87041C8050DD579688A
:1038B000306A21F4405101437960316AB1F5405FCB
:1038C00003D1206840F4003020603168880505D5B8
:1038D000B968706A890840EA8101B96031684805B1
:1038E00005D5B968B06A21F018010143B9603168A3
:1038F000080505D5B968F06A21F0C0010143B96037
:103900003168C80405D5B968306B21F440610143C2
:10391000B960316888040DD5B968706B21F4E04155
:103920000143B960716BB1F5005F03D1206840F4C9
:10393000803020603168480458D5D7F81090B06BBB
:103940004FF0000809F4407981454FD0E16E4807F7
:103950000AD4E16E4FF0010841F00401E166E06E27
:1039600000F0040000900098DFF8B050286840F0A4
:1039700001002860FFF748FA82462868C10707D48B
:10398000FFF742FAA0EB0A000228F6D903203FE035
:103990003869B9F1000F20F4407009D0B9693A696B
:1039A00042F480323A613A6922F480323A61B96174
:1039B000B16B01433961DFF8681011EA00090ED0DC
:1039C000FFF722FA0546386910EA490F07D1FFF7D9
:1039D0001BFA401B41F289318842F4D3D6E7B8F193
:1039E000000F03D0E06E20F00400E06630680104B0
:1039F0000DD53A69F06B22F4402202433A613969ED
:103A0000F06B01F44021814218BF012000D1002059
:103A1000BDE8F687E00C0246280C0246280802465C
:103A200001000024414B19684FF6FF0200021140CB
:103A300000F4E06008433E4908431860704770B5E1
:103A40003A4B1C68C4F302230124C3F10705052D7A
:103A50002EBF0F2504FA05F56D1E1E1D072E34BF5F
:103A60000023DB1E2940994004FA03F35B1E1A4031
:103A700011430901020002D42E48815470BD2E4B1F
:103A800002F00F021A4402F8041C70BD010007D4B2
:103A9000012200F01F018A40284B400943F82020F2
:103AA000704701000BD4012200F01F018A40244B13
:103AB000400943F82020BFF34F8FBFF36F8F70474B
:103AC000401EB0F1807F07D21E49486000228A6004
:103AD0000B6843F003030B60B0F1807F8041C0436B
:103AE000C00F70471849174A04281ED8DFE800F0B5
:103AF0000811141D0300106840F0040010607047A6
:103B0000136823F004031360086820F44000086081
:103B100070471368012001E01368022023F00403BA
:103B200013600A6860F397520A6070470CED00E07A
:103B30000000FA0500E400E018ED00E000E100E01C
:103B400080E100E010E000E0E00C02462DE9F04FDB
:103B50004FF0000C8E4A8F4BDFF83C824FF00F097C
:103B600006460F46A2E0012404FA0CF414EA010010
:103B700058D04FEA4C0103258D406FEA050E7D6851
:103B800005F0030ABAF1010F1CBF05F00305022D71
:103B900013D1B568D7F80CA00EEA05050AFA01FAA8
:103BA0004AEA0505B560756825EA04047D68C5F331
:103BB000001505FA0CF52C4374603D79BC6805F0DE
:103BC0000305032D08BF012C05D0F5688C400EEAD3
:103BD00005052C43F4603C7904F00304022C14D155
:103BE0004FEADC0406EB8404D4F820A04FEA8C05ED
:103BF00005F01C0509FA05FB2AEA0B0AD7F810B0F4
:103C00000BFA05F545EA0A05256234680EEA040553
:103C10003C7904F0030404FA01F129433160796826
:103C200011F4403F40D04FEA9C01DFF870A158F8F2
:103C300021E04FEACC040AEA962A04F0180409FAB3
:103C400004F52EEA05050AFA04F444EA050E48F8DC
:103C500021E0D3F800E07C68C14301EA0E0EE502E2
:103C600048BF40EA0E0EC3F800E0D3F804E07C68D9
:103C700001EA0E0EA50248BF40EA0E0EC3F804E0AA
:103C8000D2F804E07C6801EA0E0EA50348BF40EAC2
:103C90000E0EC2F804E0D2F800E07C6801EA0E01E2
:103CA000E40348BF014311600CF1010C396831FA9B
:103CB0000CF07FF458AFBDE8F08F2DE9F04F0246CD
:103CC0000027344BDFF8C8804FF00F09DFF8C8A099
:103CD00053E0012000FA07FC1CEA01004CD04FEA37
:103CE000970EDFF8B8B05AF82E60FD000BEA922B61
:103CF00005F0180509FA05F426400BFA05F5AE4261
:103D000016D1D8F80050C0430540C8F80050D8F884
:103D100004600640C8F804605D6805405D601E6888
:103D2000304018605AF82E0020EA04044AF82E4069
:103D300003207C00A0401468FD0802EB850E0443BC
:103D40001460DEF82040BD0005F01C0509FA05F5F9
:103D5000AC43CEF82040D2F808E0C04300EA0E0E93
:103D6000C2F808E0546824EA0C0CC2F804C0D2F887
:103D70000CC000EA0C00D0607F1C31FA07F0A8D11B
:103D8000BDE8F08F0AB18161704781627047000021
:103D90008020024600200246602002467F7F2F00DE
:103DA000F8B504461F4D2878002100282ED01E4A61
:103DB00012681E4B1E68770702D54FF47A710DE02A
:103DC0001B4B1B6813F4400306D0B3F5800F08D0DB
:103DD000B3F5000F0ED015E04FF4FA51B1FBF0F03F
:103DE0000EE04FF47A72B2FBF0F24FF4FA43B3FBF9
:103DF000F2F107E04FF47A71B1FBF0F04FF40042BA
:103E0000B2FBF0F10846FFF75BFE08B10120F2BDFE
:103E1000002221464FF0FF30FFF711FEAC6000207A
:103E2000F2BD00BF000000200C00002010E000E008
:103E3000E00C024680B50B48016841F480710160D6
:103E40000320FFF7EFFD00F033FC0420FFF74AFEEC
:103E50000F20FFF7A5FF08B1012002BD00F0A0FC74
:103E6000002002BD0020024038B586B0142101A810
:103E7000FFF7D0FC4648016848F29105454C41F0F7
:103E800002010160026802F00202009200990268D9
:103E900042F001020260036803F0010300930099FD
:103EA0000268294642F0040202600068002200F025
:103EB00004000090009800F049F8012102910022CE
:103EC00001950392049201A92046FFF73FFE07B037
:103ED00030BD012200E0002280212E48FFF752BFB2
:103EE00010B52C4C0122102100F030F82A4800F0C7
:103EF00079FB00F055F800F027F8642000F070FC22
:103F0000012200F022F8012200F04BF8C82000F056
:103F100067FC00F019F84FF4AF7000F061FC00F09E
:103F20003FF8642000F05CFC0C24FFF7D2FF4FF454
:103F3000FA7000F055FCFFF7CEFF4FF4FA7000F076
:103F40004FFC641EF1D110BD002201212046FFF775
:103F500019BF10B5114800F045FB0E4C00F020F8D9
:103F6000642000F03DFC012200F01BF84FF42F709C
:103F700000F036FC00F014F8FFF7ABFF1E244FF4FE
:103F80007A7000F02DFC641EF9D1BDE81040A2E764
:103F90008C0C024600040242508000087480000825
:103FA00000224FF400412046FFF7ECBE18B587B061
:103FB0001C220021684600F027FC284C284820607D
:103FC000FF20E0604FF0804000217F22E0616160CF
:103FD000A26021616161A16121626162204600F0FD
:103FE0001DFC08B1FFF790FB0021009103910491A3
:103FF00005916946204600F012FD08B1FFF784FBE9
:1040000000220021204600F0C7FC08B1FFF77CFB2E
:1040100008B010BD10B590B004464022002168469B
:1040200000F0F2FB21680E4A914215D14FF4804313
:104030004FF4007100930E916846FFF7EFFB08B153
:10404000FFF762FB0748016841F400110160006856
:1040500000F400100090009810B010BD580C002023
:1040600000780046A80C024680B5002000F0F6FC5F
:1040700008B1FFF749FB00F0FDFC18B1BDE80140B5
:10408000FFF742BB01BD00002DE9F04FA3B00020B7
:104090000090DFF8E45302260027FFF721FF05F523
:1040A0001C7ADFF8D8B30FF21C480FF20449322013
:1040B00000F096FB782000F0EFF804460A2229462B
:1040C00009A800F0E7FC0146484600F08BFA00F032
:1040D000DFF809A800F0BEF909A9404600F082FA0D
:1040E00000F0D6F809A800F0B1F909A90FF2E830FC
:1040F00000F078FA00F0CCF809A800F0B6F909A9A8
:104100000FF2E83000F06EFA00F0C2F809A800F0F3
:10411000A8F909A90FF2E03000F064FA652109A8B6
:104120007F1CFFF777FBFF2C42D00A2C47D0002CD6
:1041300022D1584600F056FA00F0AAF8684600F07E
:1041400048F9009863280DD041000246713949B200
:104150000BF12C0000F046FA08E04FF0FF3023B0DE
:10416000BDE8F08F0BF15C0000F03CFAAAA000F073
:1041700039FA0BF580702CE0FBD0012C0CD0022C0E
:1041800010D0032C11D0042C18BF052C04D00A2CFD
:1041900015D0FF2C0CD015E000F017F900260BF11C
:1041A000840016E00BF1B00013E00BF1D80010E032
:1041B0000BF5947000F016FA0BF5B07009E00FF2F1
:1041C000443006E021460FF25C3000F00BFA0BF5AC
:1041D000CE7000F007FA0FF26C3000F003FAB52150
:1041E000504600F001F9002830D151460FF26830F6
:1041F00000F0F8F90FF2683100F047F820B90FF23B
:10420000683100F042F810B10FF2643118E00FF29B
:104210006C3100F03AF820B90FF2683100F035F84F
:1042200010B10FF268310BE00FF2783100F02DF889
:1042300020B90FF2783100F028F828B10FF274316C
:1042400001A800F037FC05E0012603E00BF5F8704B
:1042500000F0C8F901A800F0D3F870B900F0DEF85A
:104260000121284601F015F8012806D100F0E0F8F8
:10427000064641F2883000F0B3FA3046002E3FF493
:104280006EAF032FFFF613AF67E7504601F033BA66
:10429000652109A8FFF7BEBA2DE9F04F85B00026C9
:1042A00003968DF81060DFF8D0B18246FEF7ACFDC2
:1042B00005467349584600F052FF72487249734AE6
:1042C000029001910092724B724A73495846FF273F
:1042D0004FF47A7400F0E3FC04FB0AF4022870D176
:1042E000584600F0F9FC022865D1FEF78DFD401B11
:1042F00060A7DFF8A8814FF6FF790EE0384600F09E
:1043000071F905E0002EF9D1404600F06BF9012665
:1043100000F05BF8FEF778FD401BA04201D3CA45D0
:1043200011D103A9584600F0F6FD0228F2D10398F6
:104330006328E7D04100B1F1710149B2A2A000F0B9
:1043400051F900F042F800BF89A20121584600F05F
:104350000FFFFEF759FD401B9DF9107004E000F0BF
:1043600034F8FEF751FD401BA04201D3CA4517D1D6
:10437000584600F049FE0128F3D1584600F028FEC7
:104380000128EED1584600F0DDFD022808D07F1C40
:1043900078B20128E3D1584600F0F9FD0228DED0BA
:1043A000584600F031FE0746012818BF052808D1FD
:1043B000FEF72AFD05E0082802BF9BF8D270032F04
:1043C0001327384605B0BDE8F08F4FF47A7000F03F
:1043D00007BA014610B500F036F800F09CFD02283F
:1043E00008BF0024204610BDCAB2014610B500F037
:1043F0002AF800F034FE022808BF0024204610BD31
:10440000024610B500F01EF800F0E8FE022808BFD2
:104410000024204610BD00000D0A000010B500F079
:1044200012F800F079FF022808BF0024204610BDD2
:1044300010B500F008F800F0B9FF022808BF00240A
:10444000204610BD01210C480224704780B564222B
:10445000134902E080B51022124900F01BFB002036
:1044600002BD80B514221049F7E780B510220F492C
:10447000F3E700002E000000B8060020947B00083F
:10448000092E0008252D0008552D00083D2D000897
:10449000FF2C0008B91C0008112B0008AC7F000895
:1044A000F4060020C2060020C007002058070020A4
:1044B0004D6F64756C65204E616D653A2025730DF6
:1044C0000A00000050726F647563742049443A20FA
:1044D00025730D0A00000000465720566572736967
:1044E0006F6E3A2025730D0A00000000494D4549C2
:1044F0003A2025730D0A000049434349443A2025D8
:10450000730D0A000D0A203E3E3E2053494D20699E
:1045100073206E6F7420494E5345525445440D0A22
:104520000D0A00000D0A203E3E3E204D6F64756C62
:10453000652053494D204572726F723A2025640DF3
:104540000A00000043656C6C756C6172204F7065E9
:104550007261746F723A200025730D0A000000002A
:10456000534D4152540000003531353033000000C6
:10457000696E7465726E657400000000474C4F42AE
:10458000450000003531353032000000696E746539
:10459000726E65742E676C6F62652E636F6D2E7020
:1045A000680000004449544F0000000035313536A2
:1045B00036000000696E7465726E65742E646974ED
:1045C0006F2E7068000000000D0A5369676E616C01
:1045D000204C6576656C3A2025642064426D0D0A96
:1045E000000000000EB4C0B5024603A800210190EF
:1045F000009101AB0121044878440C30FBF7B1FD78
:1046000006BC5DF810FB00BF953B000010B5134AD7
:10461000116B01F4803181421BD01168104B21F4E1
:104620008031084310601C6832200E494443B4FBBB
:10463000F1F1491C084601E068B1401E13681C04F2
:10464000FAD540B101E031B1491E106B0304FAD52F
:1046500009B1002010BD032010BD00000C08024667
:104660000C00002040420F0000B500BF130096462A
:104670009446103928BFA0E80C50FAD85FEA417C74
:1046800028BF0CC048BF40F8042BC90728BF20F83A
:10469000022B48BF00F8012B00BD0000374801681D
:1046A000374A41F4700101603648106070470000DD
:1046B00030B53549CB693548354A03F00C03082B32
:1046C00002D00C2B07D04BE010460A68120D02F006
:1046D0000102D04044E08B6A4C6BC3F302256D1C91
:1046E00000EE105AC4F30805C4F30664641C6D1C84
:1046F00001EE104A00EE905ADC0607D58C6BC4F32D
:10470000CC0401EE904AFBEEE91A01E0DFED1A1A43
:1047100003F00303022B02D0032B03D00AE002EEC6
:10472000100A09E00868000D00F00100C24002EE26
:10473000102A01E09FED102AB8EE422AB8EE400A96
:10474000F8EE600A82EE000A70EEA10A20EE200A5E
:10475000F8EE410A80EE200ABCEEC00A10EE100A04
:104760000C4A1060096A00BF0BA301F00701595CF5
:10477000C840106030BD00000000000088ED00E07F
:1047800008ED00E000000008000C02460024F400E0
:104790000048E8010C0000200000000001020304B2
:1047A00080B50E48816841F004018160816801F0A4
:1047B0000401009100990268002142F48012026015
:1047C0000068002200F48010009000984420FFF759
:1047D00036F94420BDE80240FFF758B98C0C024678
:1047E00038B50446FEF710FB054614F1010F02D060
:1047F000044908780419FEF707FB401BA042FAD3CE
:1048000031BD00BF0000002010B5044610460A4626
:104810000146204600F086FF204610BD70B50446D4
:104820000120002C49D004F12C05697821B9002021
:1048300028702046FFF7EEFB02216970DFF8506117
:104840003068C10636D4CA20B0615321B161204618
:1048500000F052F8010028D1F168DFF8380101407A
:10486000F160F268606821690243A0690A4302436B
:10487000F260E168A06841EA004171603268616AF3
:10488000A06A22F4F8520A4302433260204600F044
:1048900057F8010009D1F368226AE16923F0604307
:1048A000134362690B431343F360FF21B1610200BC
:1048B00003D100E000200121697070BD84F82D0053
:1048C00070BD70B50446324D286820F02000286085
:1048D000FEF79AFA0646286881060BD4FEF794FA8A
:1048E000801B40F2E9318842F5D32868810601D463
:1048F0000320E3E7002070BDF8B50546244C20688E
:10490000002641061AD4206840F080002060FEF79F
:104910007BFA074603E00320032685F82D00216873
:1049200048060BD4032E09D0FEF76EFAC01B40F2E6
:10493000E9318842F3D320684106ECD53046F2BD18
:1049400070B50446124D2868002620F080002860CB
:10495000E968880608D42046FFF7B3FFA0B103201A
:1049600084F82D0003260FE0E86820F02000E860BE
:104970002046FFF7A6FF18B1032084F82D00032678
:10498000E86840F02000E860304670BD000000009C
:104990000C780046BFFF8FFB2DE9F04100F12C069B
:1049A00030780C461546012808BF02202FD0012080
:1049B000307002217170DFF89870F86820F4806020
:1049C000F8603968480614D4FEF71EFA8046386845
:1049D00041070ED4FEF718FAA0EB080000F01BF810
:1049E000F5D33868410704D403207070002131707A
:1049F0000DE0F8680121C00845EAC005FD60BC6013
:104A0000F86840F48060F860717000203070BDE894
:104A1000F081A0EB090040F2E9318842704710B5FF
:104A20000A6848680C4B02431A608C68CA68886937
:104A3000084B144304435C601A680869496922F012
:104A4000FF12024342EA014200201A6010BD00003A
:104A50000C780046207C00461C78004610B500F01B
:104A600010F801D5012010BD136823F00403194389
:104A7000116010BD0648016841F00101016000208D
:104A80007047034A136801460020DC0770470000A6
:104A90000004034001B55AB111F8013B521E00F861
:104AA000013B03B1F8D111001CBF002200F03AFE17
:104AB00001BD00000CB430B583B00A4606A90291CE
:104AC000044600250194009502AB01A908487844EA
:104AD0001E30FBF746FB019A157000284EBF0446B6
:104AE0000198041B204603B030BC5DF80CFB00BFEE
:104AF0000FC9FFFF70B5024615780023002400207F
:104B00002D2D0AD10123521C012406E012F8016B5D
:104B10000A25641C05FB006030381578303D0A2DED
:104B2000F4D301B10C7003B1404270BD0023814247
:104B30003CBF4FF0FF331B1A591A4018101870472A
:104B40002DE9F24F82460AF5B2709CB04168934657
:104B50001C46269F884701900BF10F024FF47A50B4
:104B600042434FF4E131002692FBF1F0B84238BFE6
:104B7000384626900025DFF8EC780DF13C090DF160
:104B8000080868206843391D29F815600844FCF7B7
:104B9000C3FA28F815006D1C192DF2DB5FEA0B0033
:104BA00008BF002C51D04FF480710AF5B670FEF7A3
:104BB00031FE0AF5B27A02E0521C192A1ADBDAF841
:104BC000040080470146269A0198FFF7AFFF0028AE
:104BD00036DDDAF80010684688470028EFD19DF8E6
:104BE00000001C998855761C36B25FEA0B0224D16E
:104BF0000022682101FB02F039F812E09DF800C0A4
:104C00003B189E449EF80450AC451CBF002529F873
:104C1000125039F812509DF800E02B441B799E4544
:104C2000CAD16D1C29F8125038F81230ADB29D422D
:104C3000C2D338580442BFD00BE05E45BFDB04E06E
:104C4000BBF1000F03D0002E01DD304601E04FF034
:104C5000FF301DB0BDE8F08F2DE9FC4105460C008A
:104C600016461F466FF0010808BF4FF4AF7400F0FE
:104C7000B2FAD5F8602181B23046904700280BD4B3
:104C8000C820FFF7ADFD00943B46002205F5B67144
:104C90002846FFF755FF80464046BDE8F681F0B54F
:104CA00070B10C000CD014000AD01C0008D0059C78
:104CB000250005D0069D2E0002D0079E370001D1A9
:104CC0004020F0BD00F5A87001604260836004617F
:104CD0004561C6600220F0BD2DE9FC4780460020FA
:104CE000202788F83B010025002200230A214143A8
:104CF000414401F59F71401C0A704B704D808A80C1
:104D0000CB800028F2DD08F5A874E06880472168B0
:104D10008847002840F0F380A0694025002680479E
:104D200082460FF25C79A069804701464FF4FA721F
:104D30005046FFF7FBFE002808D542234A4600F004
:104D4000E6F80546A069761C8047824670B20A28BC
:104D50005DDA022DE7D108F5A471404600F0B9F9FB
:104D6000054642230FF2207200F0D1F8054342239A
:104D70000FF21C7200F0CBF8054342230FF21872B9
:104D800000F0C5F8284340F0020008F5B6750FF2B0
:104D9000102A022843D142230FF2087200F0B7F81C
:104DA000022806D100F0AFF801460A224046FFF77C
:104DB00071FE42230FF2F86200F0A9F8022807D131
:104DC00000F0A1F80146322208F10A00FFF762FE66
:104DD00042230FF2E86200F09AF8022807D100F0AF
:104DE00092F80146642208F13C00FFF753FE42238B
:104DF0000FF2D46200F08BF8022810D100F083F893
:104E00000146322208F1A000FFF744FE09E0022D1E
:104E1000A1D0DFF85406FFF7E5FB04275BE002288A
:104E200059D1A06980470646A1698847801BB0F523
:104E3000FA6FF9D348F2420423460FF2986241F226
:104E40007C5100F066F8022831D10FF294612846B7
:104E500000F051FC00283ED0FF2088F8D200234605
:104E60000FF28C6200F053F8022807D100F04BF8E3
:104E70000146322208F1D600FFF70CFE42230FF262
:104E80007C6200F044F802280FD100F03CF83A218F
:104E9000FCF708F918B110F8011F2029FBD00146D2
:104EA000322208F58470FFF7F5FD022713E0B0F514
:104EB000004F10D14FF47A70009001230022294650
:104EC0004046FFF73DFE01A908F26D10FFF712FE04
:104ED00088F8D200082748F242030FF22C6244F20D
:104EE000740100F016F8022818BF20274FF01E08A2
:104EF0001E20FFF775FCB8F10108F9D100E010277A
:104F00003846BDE8F6875146284600F015BC4FF4F8
:104F1000AF714046A0E67CB500F050F80FF2F452B5
:104F20004FF4AF71FFF798FE0646022E08D10FF23C
:104F3000F05100F090F86946801DFFF7DBFD286016
:104F4000304676BD7CB5044694F8D2004025FF2853
:104F50001BD148F242030FF2D052DFF8101500F0D7
:104F600096F9022810D04FF47A7004F5B6760090C6
:104F70000123002231462046FFF7E2FD31460FF2C1
:104F8000B850FFF72FFB00E00225284676BD1CB580
:104F900000F015F80FF2B052DFF8D41402E0000070
:104FA0000D0A0000FFF758FE022806D04FF47A7071
:104FB0000090012300F007F8402016BD0D4604467E
:104FC00048F242037047002204F5B6712046B7E567
:104FD0003EB500F035F815D148F242030FF2745295
:104FE00000F073F802280DD10FF2745100F033F87D
:104FF00040B16B4601AA0FF2705100F0C3FB0228CA
:1050000008BF009DE8B23EBD3EB500F019F815D1CD
:1050100048F242030FF2605200F057F802280DD117
:105020000FF2605100F017F840B16B4601AA0FF281
:105030005C5100F0A7FB022808BF009DE8B23EBD0E
:10504000002104460191009194F8D200FF25FF2829
:1050500070470FF2485104F5B67000F04CBB2DE9D3
:10506000F0410D461646DFF8087448F2420804463F
:1050700043460FF2D4423946FFF7EEFD43460FF2A6
:105080002452394600F003F90746022F16D1FFF7E4
:10509000E0FFC11D00F05FF80FF258684146FFF7CE
:1050A00033FF022404E04146002000F045FB641E6B
:1050B00038B1002CF7D1014600F04DF83846BDE874
:1050C000F0814027FAE7422342464FF4AF71204671
:1050D000C2E5F8B50C4642230FF2D4424FF4AF714B
:1050E0000546FFF7B9FD05F5B67602280AD10FF29D
:1050F000CC41304600F0FFFA0021801DFFF7FAFC9A
:10510000C5F8480142230FF2BC424FF4AF71284664
:10511000FFF7A2FD0546022D1BD10FF2B441304628
:1051200000F0E9FA861D00213046FFF7E3FC074650
:105130000021B01CFFF7DEFCFFB2C0B2022F04D189
:10514000022814BF0120032002E0022818BF00201B
:1051500060602846F2BD32462846FFF79BBC08B186
:105160000A0001D140207047C0F868110220704742
:105170002DE9FF4100F02CF8DFF8F88200F11A0168
:1051800000962B460FF25042404600F00FFBFFF70F
:105190009AFF07460FF25C420D21404600F006FBE5
:1051A000FFF791FF022F0FD179A000210391029008
:1051B000019000962B46B04A4FF48071404600F0B3
:1051C000F5FAFFF780FF0746384604B0BDE8F081E6
:1051D000044616460D463046FBF79EBF2DE9F041CA
:1051E000FFF7F6FFA34F00F1190133460FF2144207
:1051F000384600F0DBFA42233A46FFF766FF0646E0
:10520000022E2FD194F83B01022827DC2B460FF207
:1052100010421821384600F0C9FADFF8508200F039
:1052200033F800F022F8022E18D10FF204421821B0
:10523000384600F0BBFA00F027F800F016F8022E0E
:105240000CD100F01CF808B940200CE0401C00F024
:1052500071FB00F00EF8401C84F83B014FF4FA702B
:10526000FFF7BEFA3046BDE8F08106460A20FFF798
:10527000B7BA04F23B11485594F83B0170472C2112
:1052800004F5B670FBF70EBF42233A46414620466E
:10529000E2E42DE9FE4305460E46764C0FF29032CD
:1052A0000B21204600F082FA422322466F4928460D
:1052B000FFF7D2FC02282CD169A7394605F5B67054
:1052C00000F03AFA04460FF27C380FF2703904E02D
:1052D0003946002000F030FA0446D4B14946204651
:1052E00000F009FA0028F3D00021019100916B46EB
:1052F00001AA4146204600F045FA022804BF019861
:10530000B042E5D10099AA1982F83B110098C0B2C9
:1053100000E0FF20BDE8FE832DE9F04190B0044697
:1053200042230FF2303251494025FFF795FC022805
:1053300029D104F5B6700FF22C370FF23C381CE07F
:105340002221FBF7AFFE060015D02221701CFBF7CF
:10535000A9FE04000FD0841B641E3F2C88BF3F248D
:105360002246711C6846FFF795FB002069460855E8
:105370003846FFF737F905F10A00414600F0BBF95E
:105380000500DDD10225284610B0BDE8F0810000FF
:10539000000000000246002003E02C2908BF401C4A
:1053A000521C11780029F8D1704700002DE9F04710
:1053B0000446304DADF1300DB2A21C21284600F05C
:1053C000F5F942232A46FFF780FE0546022D43D118
:1053D000FDF71AFD002106460B91069105910A91F1
:1053E000099108910791002704F5B67A0FF2CC28AD
:1053F0000FF2B02923E04FF47A7000901F4B002287
:1054000051462046FFF79CFB5046FFF7C3FF062896
:1054100015D107A8049008A909AA0AAB05A8039109
:1054200002920193009006AB0BAA4946504600F049
:10543000A9F9069A059940460127FFF7D3F8FDF729
:10544000E3FC801B44F274018842D4D327B900BF27
:10545000A2A0FFF7C7F8402528460CB0BDE8F087AA
:105460000D0A00003C720008B87E0008606102006E
:1054700090D60200E00900202C80000810000800EF
:1054800041540D0A00000000415456310D0A00003D
:10549000415445300D0A000041542B434D45453DD4
:1054A000310D0A0041542B43474D490D0A000000BD
:1054B00041542B43474D4D0D0A00000041542B43EE
:1054C000474D520D0A00000041542B4347534E0DE7
:1054D0000A00000041542B4350494E3F0D0A000082
:1054E0002B4350494E3A2052454144590000000098
:1054F00041542B43494D490D0A00000041542B49AA
:10550000434349440D0A000041542B4346554E3D48
:10551000310D0A0041542B4353510D0A0000000085
:105520002B4353513A00000041542B4347415454FC
:105530003D310D0A00000000434D45204552524FB9
:10554000523A2025730D0A0041542B434F50533DCE
:10555000300D0A0041542B435245473F0D0A0000CD
:105560002B435245473A00002B435245473A2025EA
:10557000642C25640000000041542B4347524547EA
:105580003F0D0A002B43475245473A002B434752F1
:1055900045473A2025642C25640000002B434F50DA
:1055A000533A000041542B434F50533F0D0A000023
:1055B00041542B4950523F0D0A0000002B495052D4
:1055C0003A00000041542B4946433F0D0A000000B9
:1055D0002B4946433A00000041542B434744434F74
:1055E0004E543D25642C224950222C222573220D35
:1055F0000A00000041542B434744434F4E543F0D93
:105600000A00000041542B434744434F4E543D3160
:105610002C224950222C20222573220D0A00000042
:1056200041542B43474143543D312C25640D0A001E
:1056300041542B43474143543F0D0A002B434741FC
:1056400043543A002B43474143543A2025642C25C8
:105650006400000041542B434750414444523D31C3
:105660000D0A0000495020416464726573733A204A
:1056700025730D0A000000002B434750414444525B
:105680003A20000041542B5150494E473D312C22C5
:10569000382E382E382E38222C31302C31300D0A4D
:1056A000000000002025642C25642C25642C256432
:1056B0002C25642C25642C256400000050494E479D
:1056C00020526573756C743A202564206F757420C0
:1056D0006F662025640D0A0D0A00000050494E47F0
:1056E00020526573756C743A204E4F4B0D0A0D0AAB
:1056F000000000002C0070B50D462C7834B970BD48
:1057000011F8013F1678B34206D0401C2146FBF742
:10571000C9FC28B101462A4612F8013F002BEFD1FF
:1057200070BD00004018491C1CBFB1F1010100F818
:10573000012DF9D17047000038B504000D460BD09B
:105740002946204600F0FDF80444207848B90C486A
:1057500000210160002032BD09490C68002CEFD106
:1057600032BD2946204600F0FDF82118087810B116
:10577000002201F8012B02480160204632BD00BF23
:10578000880C00200DB4C0B50A4604A80021019081
:10579000009101AB03A9044878440C3000F01CF9D7
:1057A00006BC5DF810FB00BF13B9FFFF08B438B5A5
:1057B00085B009AC00250494039500290EBF01951E
:1057C0000190491E0291009504AB01A90748784455
:1057D0001A30FAF7C6FC019901B10D70002858BFC4
:1057E000039806B030BC5DF808FB00BFC3BBFFFFE9
:1057F0002DE9F84F84B00E4617460BB100221A600F
:105800000446A04601E008F1010898F8000000F005
:1058100079FF0028F7D198F800002D2816BF2B2813
:1058200018F8015B2B25002F019603D4012F01D01E
:10583000252F03DB002E56D0346054E0002F0CDD02
:10584000102F04BF98F80000302802BF98F801001C
:1058500040F02000782811D10CE098F800003028A2
:1058600018BF0A270AD198F8010040F020007828D4
:1058700003D1102708F1020800E00827CDF80C80BA
:1058800001E008F1010898F800003028F9D0064E30
:105890007E4414364FF0000906F12800CDF8088048
:1058A000CA468DF800000CE07025000001469DF806
:1058B0000000081ACA465FFA80FB07FB09B908F125
:1058C000010898F8000000F027FF01463A4606F16B
:1058D0002800FBF72BFC0028E8D10399414504D1AF
:1058E000019800B10460002020E00299F05DA8EB6F
:1058F0000101091A002910D406DCB9EB0B0103D30E
:10590000B1FBF7F0504508D0AFF30080049808B120
:10591000012101604FF0FF3903E02D2D08BFC9F1CF
:105920000009019808B1C0F80080484605B0BDE8FC
:10593000F08F04E000E000000A220021F9E70023D4
:1059400056E770B4044600E0641C23783BB10D4672
:105950002A7822B115F8016BB342F9D1F4E7201A85
:1059600070BC704770B4044600E0641C23783BB1FF
:105970000D462A78002AF8D015F8016BB342F8D109
:10598000201A70BC70470000034608460122C16817
:10599000491CC16000210068184703460846C168D9
:1059A0000269491C521E002A0261C16003D40068CA
:1059B0000122002118474FF0FF3070470346084688
:1059C0001146C268521E11F1010FC26002D0006878
:1059D00000221847704700002DE9F84F9AB04FF0A9
:1059E000FF34009100261B68019302920DF13F02E3
:1059F000249B8DF81F30A04603961992814613E030
:105A00000398401C0390012200980021C8470646D5
:105A100000F078FE0028F3D1324669464846FFF789
:105A2000CDFF0298411C02910298007800F06AFEB6
:105A30000028E5D1029E307820B9404500DA404682
:105A400000F034BD25280AD1701C029001782A2963
:105A500003BF401C029010F8011D002110E00398C4
:105A6000401C0390012200980021C84731788842E9
:105A7000D7D0024669464846FFF7A0FF0020DCE782
:105A80008DF81C1000210591DFF8143A0AE0059802
:105A9000984205DA00EB800601EB460130390591AA
:105AA000501C0290029A1178A1F130000A28EED31E
:105AB00006940FF6F0101178FBF7F4FA20B1029873
:105AC000401C0290401E00788DF81D009DF81D00BE
:105AD000682805D10299087868280CD1622206E06E
:105AE0006C2802BF029908786C2804D17122491CE5
:105AF0008DF81D200291029801780FF6A430FBF773
:105B0000D1FA80B90398401C03900122009800212B
:105B1000C847064600F0F6FD0028F3D13246694634
:105B20004846FFF74BFF00208DF81E0002980178D1
:105B3000253939D01C3900F09C80091F022940F218
:105B40009880133900F01083C91E1FD0891F00F000
:105B50009080891E00F08F84491E00F00583491E45
:105B6000022940F28680091F00F0FE82491F3ED0C4
:105B7000491E012940F2F882091F35D0891E00F024
:105B8000F382C91E00F0F08200F080BC224600F0D3
:105B900073BC2498002800F07A8416F1230F40F09B
:105BA0007684204600F082BC0398401C03900122BA
:105BB0000098C8470646252E0CD1B8F1000F48BF03
:105BC0004FF000089DF81E0000283FF42AAF08F1AE
:105BD000010826E7324669464846FFF7EFFE16F110
:105BE000010F40F05384AAE3012200F045BC9DF868
:105BF0001C000028E1D19DF81D0062282DD06828E6
:105C000011D06A281BD06C2801D0712817D00199B7
:105C100051F8040B019118B90FF68C2000F027BC45
:105C200003990160C9E7019951F8040B019118B972
:105C30000FF6742000F01BBC03990180BDE70199A9
:105C400051F8040B019118B90FF65C2000F00FBC5D
:105C5000039AD317C0E90023AFE7019951F8040B69
:105C6000019118B90FF6402000F001BC03990170B2
:105C7000A3E705980028D8BF6FF00040049069465C
:105C80004846FFF78AFE00260AAF2B2818BF2D28AA
:105C900007D18DF8280069464846FFF77EFE0DF1D2
:105CA0002907002530284FF00A0A16D169464846D0
:105CB000FFF773FE40F02001C9B2782902D0012518
:105CC0002946ECE030203870797048466946FFF785
:105CD00064FEBF1C4FF0100AF2E740F02001CAB288
:105CE0006E2A4CD16E2007F8010B69464846FFF733
:105CF00054FE83464BF02000C0B26128B24640F00B
:105D00008781612107F8011B48466946FFF745FE78
:105D100083464BF02000C0B26E2840F0798169467E
:105D20004846FFF73AFE282806D00246694648460C
:105D3000FFF744FE6E2052E00498401E049004D504
:105D40000398401C0390A34604E069464846FFF7C9
:105D50001BFE8346CDF820B0584600F0E7FC002833
:105D6000EAD1ABF130000A28E6D308985F28E3D0E7
:105D70008346BBF1290F40F04B816E202FE0C9B262
:105D8000692940F09C80692007F8010B6946484664
:105D9000FFF703FE83464BF02000C0B26E28B246E8
:105DA00040F036816E2107F8011B48466946FFF72F
:105DB000F4FD83464BF02000C0B2662840F02881F5
:105DC00069464846FFF7E9FD40F02001C9B269295C
:105DD00008D0024669464846FFF7F0FD662007F8FE
:105DE000010B1BE103980499401C491E00290491F2
:105DF000039005D4009801220021C847834600E0A3
:105E0000A3464BF02000C0B26E2840F001810398F9
:105E10000499401C491E00290491039005D4009860
:105E200001220021C847834600E0A3464BF0200032
:105E3000C0B2692840F0EC8003980499401C491EC8
:105E400000290491039005D4009801220021C8473D
:105E5000834600E0A3464BF02000C0B2742840F017
:105E6000D78003980499401C491E0029049103908F
:105E700005D4009801220021C847834600E0A346CC
:105E80004BF02000C0B2792840F0C280662107F8AC
:105E9000011BC3E069464846FFF776FD0121302823
:105EA00008D10498401E0490F4D50398401C039038
:105EB0002046F3E70D4611B1302107F8011B834658
:105EC0002846002505E069464846FFF75DFD834604
:105ED00001201BF1010F23D05FFA8BF2612AA8BFCA
:105EE000ABF157010ADA412AA8BFABF1370105DA55
:105EF000303A0A2A34BFABF13001FF21C9B2514513
:105F00000ED2242DBABF07F801BB6D1C761C049875
:105F1000401E0490D7D50398401C0390A346D7E7B2
:105F20008DF820000995FBF7EBFD406A01788B4561
:105F300010D107F801BB03980499401C491E0029A1
:105F40000491039005D4009801220021C84783469C
:105F500000E0A3460998E8B99DF8201005E06946DD
:105F60004846FFF711FD83460121BBF1300F09D1EF
:105F70000498761E401E0490F1D50398401C0390AF
:105F8000A346F1E7002E8DF8201003D5302107F845
:105F9000011B761C9DF82000099D05E069464846D6
:105FA000FFF7F2FC834601201BF1010F23D05FFABB
:105FB0008BF2612AA8BFABF157010ADA412AA8BFC8
:105FC000ABF1370105DA303A0A2A34BFABF13001C0
:105FD000FF21C9B251450ED2242D08DB0498401E82
:105FE0000490DBD50398401C0390A346DBE707F839
:105FF00001BB6D1CF2E7054650B14BF02000BAF131
:106000000A0FC0B234D1652834D001E083460D4672
:106010005A4669464846FFF7D1FC0DB30021397056
:106020009DF81C0000287FF4C8ADBAF10A0F0B469A
:1060300074DC32460AA800F073FC01228DF81E20A1
:106040009DF81D20019B6C2A73D153F8042B0193FA
:10605000002A6BD1DFF84404784400F5886006E23A
:106060000AA8874208BF1BF1010F40F00F8266E1CA
:106070007028CDD107F801BB0498401E049010D4BD
:106080000398401C0390012200980021C8472B2848
:1060900018BF2D2811D107F8010B0498401E049059
:1060A00004D50398401C0390204606E00398401C4A
:1060B0000390012200980021C847002104E06946AE
:1060C0004846FFF761FC0121302808D10498401EA2
:1060D0000490F4D50398401C03902046F3E70A008F
:1060E0001CBF302207F8012B002504E06946484612
:1060F000FFF74AFC0121A0F130020A2A86D2082DBE
:1061000008DB0498401E0490F0D50398401C0390CF
:106110002046EFE707F8010B6D1CF2E700220AA802
:1061200000F0FEFBB200FBF7A5F886E7C2E900012C
:1061300043E54C2A0AD153F8042B0193002AF5D1E8
:10614000DFF85803784400F5557090E11E681A1D79
:1061500001922EB9DFF84403784400F5507086E1CF
:1061600000F09AFC306028E505980028CCBF401E5E
:10617000DFF8280500280DF1200A04901BD40398AD
:10618000401C0390012200980021C8472B2818BF0B
:106190002D2814D18DF820000DF1210A03980499BF
:1061A000401C491E00290491039007D40098012245
:1061B0000021C84703E00399491C039120460021B0
:1061C000029A1278642A18BF752A0FD0692A08BF6C
:1061D00000260CD06F2A08BF082608D0702A1CBFE2
:1061E00042F02002782A02D1102600E00A26302848
:1061F0002DD104980125401E0490039805D4401C1D
:10620000039001220098C84702E0401C03902046FA
:1062100040F02001C9B2782916D1002E18BF102EE7
:106220001DD104981026401E0490039807D4401CEA
:106230000390012200980021C84700250FE0401C70
:106240000390254600274DE04EB9082607E0BEBB67
:106250000A2635E069464846FFF796FB01253028B7
:1062600008D10498401E0490F4D50398401C039074
:106270002046F3E72946CAB212B330220AF8012BAE
:106280001EE0412BA8BFA0F1370306DAA3F13002CC
:106290000A2A34BFA0F13003FF23DBB2F2B29342EB
:1062A0001ED219998A4514D30498401E049003986D
:1062B00012D4401C0390012200980021C8470121FC
:1062C00010F1010F0CD0C3B2612BDADBA0F1570340
:1062D000E3E70AF8010BE7E7401C039001212046A1
:1062E00005460F462A4669464846FFF767FBFFB258
:1062F000F7B100218AF800109DF81C0000287FF4F7
:106300005CAC02980078642818BF692869D03246CE
:1063100008A800F0CBFC01228DF81E20029A137809
:10632000702B10D1019B53F8042B01934AB99CE0C8
:1063300008A8824508BF15F1010F40F0A780264646
:10634000A5E0106039E49DF81D20622A39D0682A42
:1063500011D06A2A25D06C2A06D0712A29D0742A35
:1063600018D07A2A0FD035E0019B53F8042B019303
:10637000002AE6D179E0019B53F8042B0193002A0F
:1063800073D0108019E4019B53F8042B0193002A69
:10639000D7D16AE0019B53F8042B0193002AD0D196
:1063A00063E0019B53F8042B0193002A7FF4BEAEF7
:1063B0005BE0019B53F8042B0193002A7FF4B6AEF7
:1063C00053E0019B53F8042B0193002A4DD0107029
:1063D000FFF7F3BB019B53F8042B0193002AB0D1C4
:1063E00043E0324608A800F0B5FC01228DF81E20DB
:1063F0009DF81D20622AE4D0682ABCD06A2A1DD0EC
:106400006C2A06D0712A21D0742A10D07A2A07D09B
:1064100024E0019B53F8042B0193002A91D124E03E
:10642000019B53F8042B0193002A8AD11DE0019BA4
:1064300053F8042B0193002A83D116E0019B53F8F3
:10644000042B0193002A7FF471AE0EE0019B53F8F8
:10645000042B0193002A7FF469AE06E0019B53F8F8
:10646000042B0193002A7FF46CAF00BF9DA0FAF7C4
:1064700033FE261A05E000226946484600F03CF843
:106480000646002E3FF799ABFFF783BB0026B8F115
:10649000000F7FF5D4AAB046FFF7D1BA401B000029
:1064A000CBCCCC0C686A6C747A4C00001BB0BDE895
:1064B000F08FC9B208E003789942A4BF90F802C0F7
:1064C0008C4515DAC01CD21E032A09D343782D2B24
:1064D000F1D010F801CB8C4518BF521EF4D107E063
:1064E00042B110F8013B8B4202D0521EF9D101E0BB
:1064F00001207047002070472DE9F04F9246002799
:10650000BAF1000F83B080460E464FF0000B25D540
:10651000B068411CB160084601785E2903BF401C89
:10652000B06010F8019DB946B56828785D280CBFA9
:10653000681C28465D21FAF7B5FD002800F0A6800A
:10654000411B0091B0600098032807DB821E2D21BB
:10655000681CFAF7EBFD08B14FF0010B70690028D9
:1065600005DCBAF1000F14BF6FF00040012030616C
:10657000307F002801BF706850F8044B7060002C19
:1065800008D14FF0FF3402487844001D11E000BFED
:10659000081B0000307FA8B9F07F98B1716851F8EE
:1065A000040B7160B0F1004FC0F007804FF0FF3472
:1065B00044A0FAF791FD201A6DE0B169884288BFC6
:1065C0000846B061CDF80490CDF808B0DDF8009031
:1065D00000E00227F0683169401C491E0029316142
:1065E000F06002D54FF0FF3B38E030680122002117
:1065F000C04783461BF1010F30D0BAF1000F0CDC0D
:106600001ED50298002801980AD000284A4659460B
:10661000284612D0FFF74DFF09E000F073F806E0BE
:1066200000284A465946284603D0FAF77FFD38B17C
:1066300014E0FAF77BFD88B102E0FFF73AFF68B19A
:10664000307F0028C5D1B06938B104F801BB012101
:10665000B069B177401EB061BBE7012740465A469A
:106660003146FFF7ABF9BAF1000F01D0022F09D084
:10667000022F0FD0F80702D41BF1010F06D14FF003
:10668000FF3008E0307F28B9B06908B9002002E087
:1066900000202070012003B0BDE8F08FFEFFFF7FD7
:1066A00063436E5B000000007363616E665F733A64
:1066B0002062616420256E20617267756D656E745D
:1066C000000000007363616E665F733A206261646C
:1066D0002025632C2025732C206F7220255B2073CE
:1066E000697A65007363616E665F733A2062616404
:1066F00020696E746567657220617267756D656E7D
:106700007400000010B50446FBF7F8F90146204676
:10671000096ABDE81040084710B50446FBF7EEF9DA
:1067200001462046896ABDE81040084710B5044676
:10673000FBF7E4F9014620460969BDE81040084727
:10674000F8B52DED048B140082B041EC180B1D46FA
:1067500000F0DA8031F0004108BF002800F0D4805A
:1067600051EC180B4A00521512F1010F02D1080327
:1067700000F0CA80002C9FED689B57D56442654F9E
:106780007F4407F5C87708260CE0E00707D5D7E96E
:10679000002351EC190BFBF7BDF841EC190B640811
:1067A0000837761E002C18BF002EEED16A4651EC39
:1067B000180BFAF7F3FC009E53EC192BFAF766FF5F
:1067C0003246FAF757FD41EC180B31F0004108BF93
:1067D000002800F0828051EC180B4A00521512F18B
:1067E000010F01D1080378D0002C76D06A4651EC15
:1067F000180BFAF7D3FC009E994A9A4BFBF78AF8DC
:106800003246FAF737FD41EC180B31F0004108BF72
:10681000002862D051EC180B4A00521512F1010FFA
:1068200001D1080359D0641EE0D156E055DD394F3F
:106830007F4407F1E0070826E00707D5D7E90023E2
:1068400051EC190BFBF766F841EC190B6410083793
:10685000761E002C01DD002EEED16A4651EC180B9D
:10686000FAF79CFC2646009C53EC192BFBF752F8D8
:106870002246FAF7FFFC41EC180B31F0004108BF4B
:1068800000282AD051EC180B4A00521512F1010FC2
:1068900001D1080321D0002E1FDD6A4651EC180BF0
:1068A000FAF77CFC009C704A784BFBF733F82246E1
:1068B000FAF7E0FC41EC180B31F0004108BF00286A
:1068C0000BD051EC180B4A00521512F1010F01D1F7
:1068D000080302D0761E002EDFDC51EC180B31F0DD
:1068E000004108BF002808D051EC180B4A0052158F
:1068F00012F1010F08D1080306D1AFF300801DB1DA
:10690000286840F00100286002B051EC180BBDEC83
:10691000048BF4BDD4150000000000000000F03F1F
:106920002DE9F14D81B00C462DED028B84B09346DC
:106930005FEA030A1CBF0020CAF80000079D07A8F1
:1069400000F00BFAC11020F00800012801F0010846
:1069500032D10220009001AB07992246284600F070
:106960008DFA040008BF9FED4A0B1ED00298FAF77B
:106970004BFD022C41EC100B17DB03AF661E9FEDA5
:106980003B8B51EC100B53EC182BFAF7C3FF04466A
:1069900057F8040B0D46FAF737FD22462B46FAF757
:1069A00045FD761E41EC100BEBD1019800EB0B027C
:1069B000534651EC100B33E0022836D1009001AB66
:1069C00007992246284600F035FB040008BF9FEDDA
:1069D000300B1ED00298FAF717FD022C41EC100B79
:1069E00017DB03AF661E9FED238B51EC100B53ECAE
:1069F000182BFAF78FFF044657F8040B0D46FAF7E9
:106A000003FD22462B46FAF711FD761E41EC100BD2
:106A1000EBD1019A51EC100BFAF72CFC53465A4675
:106A2000FFF78EFE41EC100B0AE0032808BF9FED34
:106A3000130B05D004280CBF9FED120B9FED140B18
:106A4000B8F1000F05D051EC100B81F0004141EC82
:106A5000100B04B051EC100BBDEC028BBDE8FC8DAB
:106A6000436FAC642806C80A3CBF737F0000000077
:106A700065CDCD41000000000000B04100000000E5
:106A80000000F07FFFFFFFFFFFFFFF7FDD4F157569
:106A9000000000000000000001F000428B1AA3F18A
:106AA0006051B1F5801F0ADBB1F17F6F1FD242EA5E
:106AB000C102C10071F1004142EB507070470B15EB
:106AC000C3F10903212B10D2890241EA90518002BF
:106AD0000128494141F0004121FA03F0C3F12003AC
:106AE000994071F1004150417047100070476FF0BC
:106AF000000013EB103F5CBF000E42EAC05070472D
:106B00002DE9FC4F85B00C4693460BB100221A606C
:106B10000290824601E00AF1010A9AF80000FFF7AC
:106B2000F1FD0028F7D19AF800002D2818BF2B2876
:106B300007BF1AF8010B8DF800002B218DF800100B
:106B4000BBF1000F019405D4BBF1010F02D0BBF1E2
:106B5000250F04DB002C72D0029820606FE0BBF19F
:106B6000000F0DDDBBF1100F04BF9AF800003028B4
:106B700002BF9AF8010040F02000782814D10EE0FE
:106B80009AF80000302818BF4FF00A0B0CD19AF881
:106B9000010040F02000782804D14FF0100B0AF1DA
:106BA000020A01E04FF0080BCDF810A001E00AF155
:106BB000010A9AF800003028F9D0094878442030BA
:106BC0000024283000260027CDF80CA00025A04680
:106BD0008DF80100DFF80890F94409F1040919E083
:106BE0008812000001469DF80100081A5FFA80F83B
:106BF0005846A0FB06234FEAEB7100FB073301FB6D
:106C00000633344600213D4612EB080643EB0107EC
:106C10000AF1010A9AF80000FFF77EFD01465A4684
:106C200009F12800FAF782FA0028DBD104995145CE
:106C30005A4607D1019810B10199029808600020C6
:106C4000002130E0039919F80200AAEB0101091AAA
:106C500000291BD410DC0023B6EB080067EB03010E
:106C60008F4209D301D8864206D3D317FAF74EFFD5
:106C7000A94208BFA04209D0AFF30080069808B12E
:106C8000012101604FF0FF36374606E09DF8000015
:106C90002D2802D1764267EB4707019808B1C0F86A
:106CA00000A03046394607B0BDE8F08F00BF002392
:106CB00026E700002DE9F8430D0091461E4608BF67
:106CC0006D468046444600E0641C2078FFF71AFDBC
:106CD0000028F9D127782D2F18BF2B2F05D114F8B4
:106CE000010FFFF70FFD08B109E02B2733464A4695
:106CF00029462046FFF704FF2A68944205D1C5F8CB
:106D0000008000200021BDE8F4832B2F05D14FF037
:106D10000043994209D2BDE8F4832D2FFBD1B1F194
:106D2000004F12D301D801280FD3AFF300800EB16A
:106D3000012030602D2F19BF4FF0FF306FF0004160
:106D400000204FF00041BDE8F483404261EB410177
:106D5000BDE8F48300BF0023ACE72DE9F843054606
:106D60000C462E68002700E0761C3078FFF7CAFC3E
:106D70000028F9D130782D280CBF08272B2800D106
:106D8000761C307840F020016E2927D1707840F0D1
:106D90002000612802BFB07840F020006E2802D0A9
:106DA0002E68002746E0F61CB046042798F800003D
:106DB00028283FD118F8019F4846FFF7B7FC002864
:106DC000F8D1A9F130000A28F4D398F800005F2820
:106DD000F0D029282ED108F101062BE069292CD109
:106DE000707840F020006E2802BFB07840F020009C
:106DF000662802D02E6800271CE016F8030F40F02A
:106E0000200047F00307692802BF707840F0200097
:106E10006E280FD1B07840F02000692802BFF078CA
:106E200040F02000742805D1307940F02000792806
:106E300008BF761DF4B126601CE0302802BF7078D0
:106E400040F02000782813D1B01C01782E2908BF0B
:106E5000401C0078A0F16101062921BFA0F1410288
:106E6000062A30380A2803D2B61C47F0020701E090
:106E700047F001072E603846BDE8F2832DE9F14F57
:106E80008CB04FF00008169D05EBC5059246C34631
:106E90002D2DC8BF2D25C3F800B0C3F804B0D946C6
:106EA00002E0491C4FF0010908783028F9D000248D
:106EB00011E01868401C18600A78302A08D04FF09A
:106EC000010805E0AC42F4DA30380DF80400641C27
:106ED000491C4FF001090878A0F130020A2AF1D3C9
:106EE0000F461E46FAF70CFE406A39780278914246
:106EF00008BF7F1C002C48460ED1397830290BD1B1
:106F00003068401E30607F1C0120F6E7302918BF32
:106F10004FF001087F1C01203978A1F130020A2AC4
:106F20000AD2AC42F2DAA1F130000DF80400641C80
:106F30003268521E3260EDE7B8F1000F0DD00DF14E
:106F4000FF314A5D521C4A5507E00DF1FF32115DD9
:106F500049B93268521C3260641E002CF5DC04BF53
:106F60008DF800B00124002856D0092394FBF3F3D8
:106F7000C4F1090903EBC3034B44092193FBF1F16D
:106F8000002201EBC101591A1AD04FF0010B17E092
:106F900056F82B1001EB810105EB410146F82B104F
:106FA0000CE0092193FBF1F101EBC1011DF8025046
:106FB000591AEDD10BF1010B46F82B505B1C521CFA
:106FC000A242EEDB397841F02001652924D139460F
:106FD00017F8012F2B2A16BF2D2A17F8014B2B2447
:106FE00000220023124D08E0AB4204DA03EB8302D7
:106FF0000CEB4203303B7F1C012297F800C0ACF140
:10700000300EBEF10A0FEFD32D2C08BF5B4234685F
:107010001B19336002B90F46BAF1000F03D000B953
:107020000C9FCAF8007058460DB0BDE8F08F00BF45
:1070300000E1F5052DE9F14F8CB09146DDF858805F
:10704000C8EBC8084FF0000AB8F1230FC8BF4FF0D3
:107050002308C3F800A0C3F804A0002701E0491CDE
:10706000012708783028FAD068A201925FF0000466
:107070006CA200920DF1080B0D461E460EE0306822
:10708000401C306008E0A045F9DB019A0099801AA5
:10709000085C0BF80400641C6D1C012795F80010B7
:1070A0005AA01622FAF742F80028ECD1FAF728FD88
:1070B000406A29780278914208BF6D1CB4B92878DB
:1070C000302813D13168491E31606D1C0127F6E765
:1070D000A04509DB019A0099801A085C0BF80400AE
:1070E000641C3168491E31606D1C01272978162205
:1070F00046A0FAF71BF80028EAD1A04517DA1BF8DA
:107100000810072906DD0DF1070111F80820521CAF
:1071100001F8082044463268521C326007E00DF145
:107120000702115D49B93268521C3260641E002C9E
:10713000F5DC04BF8DF808A0012431688900002F18
:10714000316055D0072394FBF3F3C4F1070BC3EB75
:10715000C3035B44072193FBF1F10022C1EBC101A2
:10716000591A19D04FF0010A16E056F82A100BEB05
:10717000011046F82A000DE0072102A893FBF1F167
:10718000C1EBC10110F802B0591AEED10AF1010A9F
:1071900046F82AB05B1C521CA242EDDB297841F074
:1071A0002001702924D1294615F8012F2B2A16BF5A
:1071B0002D2A15F8014B2B2400220023124808E049
:1071C000834204DA03EB83020CEB4203303B6D1C79
:1071D000012295F800C0ACF1300EBEF10A0FEFD3DA
:1071E0002D2C08BF5B4234681B19336002B90D4671
:1071F000B9F1000F03D007B90C9DC9F800505046F3
:107200000DB0BDE8F08F000000E1F50530313233FC
:1072100034353637383961626364656641424344C8
:1072200045460000000102030405060708090A0B91
:107230000C0D0E0F0A0B0C0D0E0F000010000000BD
:107240004F4B0D0A0000000000000000000000008D
:10725000000000000000000000000000000000002E
:10726000000000000000000000000000000000001E
:10727000000000000000000000000000000000000E
:1072800000000000000000000000000000000000FE
:1072900000000000000000000000000000000000EE
:1072A00000000000080000003E0000000000000098
:1072B00000000000000000000000000000000000CE
:1072C00000000000000000000000000000000000BE
:1072D00000000000000000000000000000000000AE
:1072E000000000000000000000000000000000009E
:1072F000000000000000000000000000000000008E
:10730000000000000000000000000000004000003D
:107310004349505258474554000000000000000007
:10732000000000000000000000000000000000005D
:10733000000000000000000000000000000000004D
:10734000000000000000000000000000000000003D
:10735000000000000000000000000000000000002D
:10736000000000000000000000000000000000001D
:10737000000000000000040043495053454E440003
:1073800000000000000000000000000000000000FD
:1073900000000000000000000000000000000000ED
:1073A00000000000000000000000000000000000DD
:1073B00000000000000000000000000000000000CD
:1073C00000000000000000000000000000000000BD
:1073D00000000000000000000000000000000200AB
:1073E000504F574552454420444F574E0D0A000018
:1073F000000000000000000000000000000000008D
:10740000000000000000000000000000000000007C
:10741000000000000000000000000000000000006C
:10742000000000000000000000000000000000005C
:10743000000000000000000000000000000000004C
:1074400000000000000009005244590D0A0000002D
:10745000000000000000000000000000000000002C
:10746000000000000000000000000000000000001C
:10747000000000000000000000000000000000000C
:1074800000000000000000000000000000000000FC
:1074900000000000000000000000000000000000EC
:1074A000000000000000000000000000800000005C
:1074B000636C6F7365642200000000000000000030
:1074C00000000000000000000000000000000000BC
:1074D00000000000000000000000000000000000AC
:1074E000000000000000000000000000000000009C
:1074F000000000000000000000000000000000008C
:10750000000000000000000000000000000000007B
:107510000000000000010000434950525847455404
:107520003A53554343455353000000000000000008
:10753000000000000000000000000000000000004B
:10754000000000000000000000000000000000003B
:10755000000000000000000000000000000000002B
:10756000000000000000000000000000000000001B
:107570000000000000000000000000000002000009
:10758000696E636F6D696E672066756C6C220000B2
:1075900000000000000000000000000000000000EB
:1075A00000000000000000000000000000000000DB
:1075B00000000000000000000000000000000000CB
:1075C00000000000000000000000000000000000BB
:1075D00000000000000000000000000000000000AB
:1075E0000000000000040000696E636F6D696E6743
:1075F0002200000000000000000000000000000069
:10760000000000000000000000000000000000007A
:10761000000000000000000000000000000000006A
:10762000000000000000000000000000000000005A
:10763000000000000000000000000000000000004A
:107640000000000000000000000000000008000032
:1076500070647064656163742200000000000000C3
:10766000000000000000000000000000000000001A
:10767000000000000000000000000000000000000A
:1076800000000000000000000000000000000000FA
:1076900000000000000000000000000000000000EA
:1076A00000000000000000000000000000000000DA
:1076B00000000000001000002B4D444E534749507D
:1076C0003A00000000000000000000000000000080
:1076D00000000000000000000000000000000000AA
:1076E000000000000000000000000000000000009A
:1076F000000000000000000000000000000000008A
:107700000000000000000000000000000000000079
:107710000000000000000000000000004000000029
:107720004552524F520D0A000000000000000000B8
:107730000000000000000000000000000000000049
:107740000000000000000000000000000000000039
:107750000000000000000000000000000000000029
:107760000000000000000000000000000000000019
:107770000000000000000000000000000000000009
:1077800000000000008000002B434D452045525270
:107790004F523A20000000000000000000000000EE
:1077A00000000000000000000000000000000000D9
:1077B00000000000000000000000000000000000C9
:1077C00000000000000000000000000000000000B9
:1077D00000000000000000000000000000000000A9
:1077E0000000000000000000000000000020000079
:1077F0004552524F520D0A000000000000000000E8
:107800000000000000000000000000000000000078
:107810000000000000000000000000000000000068
:107820000000000000000000000000000000000058
:107830000000000000000000000000000000000048
:107840000000000000000000000000000000000038
:1078500000000000020000004F4B0D0A0000000075
:107860000000000000000000000000000000000018
:107870000000000000000000000000000000000008
:1078800000000000000000000000000000000000F8
:1078900000000000000000000000000000000000E8
:1078A00000000000000000000000000000000000D8
:1078B00000000000000000000000000020000000A8
:1078C0004F50454E3A00000000000000000000004C
:1078D00000000000000000000000000000000000A8
:1078E0000000000000000000000000000000000098
:1078F0000000000000000000000000000000000088
:107900000000000000000000000000000000000077
:107910000000000000000000000000000000000067
:10792000000000000400000072656164790D0A0027
:107930000000000000000000000000000000000047
:107940000000000000000000000000000000000037
:107950000000000000000000000000000000000027
:107960000000000000000000000000000000000017
:107970000000000000000000000000000000000007
:1079800000000000000000000000000000000800EF
:107990000D0A0D0A4F4B000000000000000000001F
:1079A00000000000000000000000000000000000D7
:1079B00000000000000000000000000000000000C7
:1079C00000000000000000000000000000000000B7
:1079D00000000000000000000000000000000000A7
:1079E0000000000000000000000000000000000097
:1079F00000000000100008000D0A0D0A0000000041
:107A00000000000000000000000000000000000076
:107A10000000000000000000000000000000000066
:107A20000000000000000000000000000000000056
:107A30000000000000000000000000000000000046
:107A40000000000000000000000000000000000036
:107A5000000000000000000000000000100009000D
:107A60002B5150494E473A20000000000000000012
:107A70000000000000000000000000000000000006
:107A800000000000000000000000000000000000F6
:107A900000000000000000000000000000000000E6
:107AA00000000000000000000000000000000000D6
:107AB00000000000000000000000000000000000C6
:107AC000000000002000090052445900000000009E
:107AD00000000000000000000000000000000000A6
:107AE0000000000000000000000000000000000096
:107AF0000000000000000000000000000000000086
:107B00000000000000000000000000000000000075
:107B10000000000000000000000000000000000065
:107B20000000000000000000000000000100000054
:107B30000D0A00000000000000000000000000002E
:107B40000000000000000000000000000000000035
:107B50000000000000000000000000000000000025
:107B60000000000000000000000000000000000015
:107B70000000000000000000000000000000000005
:107B800000000000000000000000000000000000F5
:107B9000000000005375636365737366756C20495C
:107BA0006E697469616C697A6174696F6E206F6661
:107BB00020746865204D6F64756C650D0A0D0A00B0
:107BC0005369676E616C205175616C697479204CE2
:107BD0006576656C2025642064426D202847534DEE
:107BE00020466F726D61743A20256C64290D0A007D
:107BF0005369676E616C205175616C697479204CB2
:107C00006576656C206E6F7420646574656374615D
:107C1000626C650D0A0000000D0A203E3E3E204DBC
:107C20006F64756C652052656769737472617469FD
:107C30006F6E205375636365737366756C0D0A0D03
:107C40000A0000000D0A203E3E3E204D6F64756C18
:107C50006520526567697374726174696F6E205430
:107C60007279696E670D0A0D0A0000000D0A203E48
:107C70003E3E204D6F64756C652052656769737474
:107C8000726174696F6E2044656E6965640D0A0DDA
:107C90000A0000000D0A203E3E3E204D6F64756CC8
:107CA0006520526567697374726174696F6E2046EE
:107CB00061696C65640D0A0D0A0000000D0A203E22
:107CC0003E3E204D6F64756C6520415420436F6DBE
:107CD0006D756E69636174696F6E204572726F7243
:107CE00020776974682074686520446576696365E7
:107CF0000D0A0000203E3E3E204465766963652003
:107D00006D6967687420626520646973636F6E6E65
:107D10006563746564206F722077726F6E676C792B
:107D200020636F6E6E65637465640D0A0D0A000052
:107D3000203E3E3E20506C6561736520636865633C
:107D40006B206966207468652053494D2069732053
:107D5000696E73657274656420616E642076616C0F
:107D600069642C2069662063726564656E7469615C
:107D70006C7320617265206F6B2C206574632E0D0F
:107D80000A0D0A000D4661696C656420746F2067F6
:107D90006574207468652063757272656E74206303
:107DA000656C6C756C6172206F70657261746F7256
:107DB000206E616D650D0A0D0A000000203E3E3EFA
:107DC00020496E697469616C697A65204D5154541B
:107DD00020436F6E6E656374696F6E0D0A0D0A0045
:107DE0004E6F204E6574776F726B20436F6E6E65B9
:107DF0006374696F6E20417661696C61626C6520A5
:107E00002D2D2050726F6365656420746F204D6F57
:107E1000646520320D0A000000002115110E0D0CC2
:107E20000B0B0A0A090909090908080808080808C3
:107E300007070707070707070707070707000000E7
:107E400030313233343536373839616263646566D0
:107E50006768696A6B6C6D6E6F707172737475763A
:107E60007778797A0000000000004129211C191759
:107E70001615141312121111111010100F0F0F0FED
:107E80000E0E0E0E0E0E0E0D0D0D0D0D0D00000042
:107E90003031323334353637383961626364656680
:107EA0006768696A6B6C6D6E6F70717273747576EA
:107EB0007778797A000000004661696C20746F2041
:107EC00041542053594E432C2061667465722073CF
:107ED00065766572616C20617474656D7074730D84
:107EE0000A00000000000000000000000000244024
:107EF0000000000000005940000000000088C3405E
:107F00000000000084D797410080E03779C34143E7
:107F1000176E05B5B5B89346F5F93FE9034F384DEF
:107F2000321D30F94877825A3CBF737FDD4F15759B
:107F300080B50D49794430310C4A7A442E32914251
:107F400003D00B49AFF3008002BD8DF80000012281
:107F500069460120FAF72AFF012802D19DF80000A6
:107F600002BD4FF0FF3002BD9880FFF79480FFF70D
:107F70009000002030B4002512E050F8042BD30705
:107F800044BF4A44521E091F042942F8045BFAD236
:107F900013468C0744BF15809B1CC90748BF1D7042
:107FA00050F8041B0029E8D130BC70475369676E54
:107FB000616C206973206E6F74206B6E6F776E201A
:107FC0006F72206E6F742064657465637461626C97
:107FD00065207965742E2E2E200000007363616E7B
:107FE000665F733A2062616420666C6F6174696ECB
:107FF000672D706F696E7420617267756D656E7440
:108000000000000010B5074979441831064C7C4443
:10801000163404E00A68081D114488470146A1424D
:10802000F8D110BD080100002401000041542B517B
:1080300049435347503D25642C312C222573222C73
:10804000222573222C222573222C25640D0A000080
:10805000202D2D2D205155454354454C2045473961
:108060003120506F776572205570202D2D2D0D0A0F
:1080700000000000202D2D2D205155454354454C26
:108080002045473931205368757420446F776E203E
:108090002D2D2D200D0A00007363616E665F733A0B
:1080A000206261642025632C2025732C206F7220B0
:1080B000255B20617267756D656E7400FEE7FEE7F3
:1080C000FEE7FEE7FEE770477047704700F008B82C
:1080D0000148F9F793BE0000740B002000F008B8C7
:1080E00002494A68087882184A60704700000020F8
:1080F0000349C8680A6882430A60486000F002B811
:10810000001D0C42704700004EF68851CEF200016F
:10811000086840F470000860BFF34F8FBFF36F8FA3
:108120004FF00170E1EE100A7047000049FEFFFFBA
:10813000B80B0000D800002000000000EB8EFFFF0D
:108140009C010000B40000000000002000F00DF8C9
:10815000002801D0FFF756FFAFF300800020AFF3F7
:108160000080FBF76BFA00F002F80120704700F086
:1081700001B8000007463846F9F750FDFBE700005C
:108180000548014603B4684680F30988AFF30080D0
:10819000FFF7BAFFFFF7DAFFA5EDF5FE38B50446A5
:1081A0000D462846FFF7C4FEA84218BF002420460B
:1081B00032BD000001488047014800479D46000845
:1081C000818100080000000001020304FFF7FEBFE8
:1081D000FFF7FEBFFFF7FEBFFFF7FEBFFFF7FEBFD3
:1081E000FFF7FEBFFFF7FEBFFFF7FEBFFFF7FEBFC3
:1081F000FFF7FEBFFFF7FEBFFFF7FEBFFFF7FEBFB3
:10820000FFF7FEBFFFF7FEBFFFF7FEBFFFF7FEBFA2
:10821000FFF7FEBFFFF7FEBFFFF7FEBFFFF7FEBF92
:10822000FFF7FEBFFFF7FEBFFFF7FEBFFFF7FEBF82
:10823000FFF7FEBFFFF7FEBFFFF7FEBFFFF7FEBF72
:10824000FFF7FEBFFFF7FEBFFFF7FEBFFFF7FEBF62
:10825000FFF7FEBFFFF7FEBFFFF7FEBFFFF7FEBF52
:10826000FFF7FEBFFFF7FEBFFFF7FEBFFFF7FEBF42
:10827000FFF7FEBFFFF7FEBFFFF7FEBFFFF7FEBF32
:10828000FFF7FEBFFFF7FEBFFFF7FEBFFFF7FEBF22
:10829000FFF7FEBFFFF7FEBFFFF7FEBFFFF7FEBF12
:1082A000FFF7FEBFFFF7FEBFFFF7FEBFFFF7FEBF02
:1082B000FFF7FEBFFFF7FEBFFFF7FEBFFFF7FEBFF2
:1082C000FFF7FEBFFFF7FEBFFFF7FEBFFFF7FEBFE2
:1082D000FFF7FEBFFFF7FEBFFFF7FEBF4301000140
:1082E000221008F0050724F400D21800080452FFF9
:1082F00001E32A1414200400008A1600084C1148D7
:1083000022204B2002C71A00080852C10812DD08BB
:1083100012C50452F110E101618810070204010145
:10832000080C00205804520804211B610812D46074
:0683300052C064F10B01D4
:0400000508008181ED
:00000001FF
